S01700005333324B5F426F6F746C6F616465722E73726563A0
S1130000007000201104000059040000590400008D
S113001059040000590400005904000000000000C5
S1130020000000000000000000000000590400006F
S11300305904000000000000590400002566000077
S1130040553B00005F3B0000693B0000733B000030
S11300507D3B0000873B0000913B00009B3B000080
S1130060A53B0000AF3B0000B93B0000C33B0000D0
S1130070CD3B0000D73B0000E13B0000EB3B000020
S1130080F53B000059040000590400005904000025
S113009059040000590400005904000059040000E8
S11300A0834800008D480000C34B0000CD4B000086
S11300B0D74B000059040000590400005904000003
S11300C059040000590400005904000059040000B8
S11300D059040000590400005904000059040000A8
S11300E05904000059040000590400005904000098
S11300F05904000059040000590400005904000088
S11303F0590400005904000059040000FFFFFFFFE6
S1130400FFFFFFFFFFFFFFFFFFFFFFFFFE7FFFFF79
S113041072B64FF000014FF000024FF000034FF0AE
S113042000044FF000054FF000064FF00007B846F7
S1130430B946BA46BB46BC4604488546044880478C
S11304400448804762B606F013F9FEE70070002006
S1130450B11E0000ED1E0000FFF7FEBF53B94AB9FC
S1130460002908BF00281CBF4FF0FF314FF0FF30B8
S113047000F07EB9ADF1080C6DE904CE00F006F889
S1130480DDF804E0DDE9022304B070472DE9F0470C
S1130490089D04468E46002B4ED18A4294466DD95F
S11304A0B2FA82F757B1C7F1200EB94020FA0EFE16
S11304B002FA07FC4EEA010E00FA07F44FEA1C495F
S11304C0210CBEFBF9F61FFA8CF809FB16EE41EA83
S11304D00E4106FB08F38B420AD91CEB010106F11D
S11304E0FF3280F027818B4240F22481023E614436
S11304F0C91AA4B2B1FBF9F009FB101144EA014492
S113050000FB08F8A0450AD91CEB040400F1FF33F2
S113051080F00E81A04540F20B810238644440EA29
S11305200640A4EB080400267DB1FC4000232C60A7
S11305306B603146BDE8F0878B4209D9002D00F08D
S11305401481002685E8030030463146BDE8F08773
S1130550B3FA83F6002E40F090808B4202D382429D
S113056000F2FD80841A61EB030101208E46002D08
S1130570EBD085E810403146BDE8F0871AB94FF05A
S1130580010CBCFBF2FCBCFA8CF7A7BBA1EB0C037F
S11305904FEA1C421FFA8CF80126B3FBF2FE210C31
S11305A002FB1E3341EA034108FB0EF38B4208D9D8
S11305B01CEB01010EF1FF3002D28B4200F2D1801C
S11305C08646C91AA3B2B1FBF2F002FB101143EA4A
S11305D0014408FB00F8A04508D91CEB040400F111
S11305E0FF3302D2A04500F2B7801846A4EB0804FA
S11305F040EA0E4098E7C7F1200301FA07F40CFA29
S113060007FC20FA03FED9404FEA1C424EEA040ECE
S1130610B1FBF2F64FEA1E4302FB16111FFA8CF8E7
S113062043EA014306FB08F1994200FA07F40AD9A8
S11306301CEB030306F1FF3080F08C80994240F2FA
S11306408980023E63445B1A1FFA8EF1B3FBF2F019
S113065002FB103341EA034100FB08F38B4208D943
S11306601CEB010100F1FF3E70D28B426ED90238BF
S11306706144CB1A40EA06468FE7C6F1200722FA06
S113068007F8B34001FA06F448EA030320FA07FC2A
S11306904FEA134EF9404CEA040CB1FBFEF94FEA61
S11306A01C440EFB19111FFA83F844EA014109FBAB
S11306B008F48C4202FA06F200FA06FA08D959182C
S11306C009F1FF3044D28C4242D9A9F102091944FC
S11306D0091B1FFA8CFCB1FBFEF00EFB10114CEA57
S11306E0014400FB08F8A04507D91C1900F1FF31AB
S11306F02AD2A04528D902381C4440EA0940A4EB78
S11307000804A0FB02894C45C446494616D313D0BD
S113071055B1BAEB0C0364EB010404FA07F7F34098
S11307201F43F4402F606C6000263146BDE8F0871B
S11307301846F4E61646DBE6C245E9D2B8EB020CED
S113074069EB03010138E3E70846D6E7704690E712
S11307508146BDE7064676E70238644446E73046FC
S113076005E7AEF1020E61442BE72E462846ECE67F
S1130770704700BF000000000000000000000000FF
S113078001F0FF01102A2BDB10F0070F08D010F83E
S1130790013B013A8B422DD010F0070F42B3F6D142
S11307A0F0B441EA012141EA014122F007047FF05B
S11307B000070023F0E80256083C85EA010586EAB2
S11307C0010685FA47F5A3FA87F586FA47F6A5FAEE
S11307D087F68EB9EED1F0BC01F0FF0102F00702FA
S11307E032B110F8013B013A83EA010313B1F8D1A5
S11307F00020704701387047002D06BF3546033886
S1130800073815F0010F07D1013015F4807F02BFBE
S1130810013015F4C03F0130F0BC0138704700BF0F
S113082080B582B000AF786039607B68002B05D05A
S11308307B68012B02D07B68022B03D1396878686E
S113084001F0BAF900BF0837BD4680BD80B584B059
S113085000AFF860B9601346FB80FB68002B05D03D
S1130860FB68012B02D0FB68022B08D1FB881A46D7
S1130870B968F86801F0DAF9F86801F03FF900BFE7
S11308801037BD4680BD80B584B000AF78600023CA
S1130890FB817B68002B05D07B68012B02D07B6831
S11308A0022B04D1786801F001FA0346FB81FB892D
S11308B018461037BD4680BD80B582B000AF786061
S11308C00B46FB707B68002B05D07B68012B02D0A4
S11308D07B68022B04D1FB781946786801F030F963
S11308E000BF0837BD4680BD80B582B000AF7860D8
S11308F07B68002B05D07B68012B02D07B68022B20
S113090002D1786801F0FAF800BF0837BD4680BD0F
S113091080B483B000AF78600B467B8000BF0C3797
S1130920BD465DF8047B704780B487B000AF786043
S11309300B467B807B68FB600023FB827B88BB8249
S113094027E0FB685A1CFA601B781B021AB2B7F93D
S1130950163053401BB2FB8208237B8213E0B7F9A5
S11309601630002B09DAFB8A5B001BB283F4815337
S113097083F001031BB2FB8202E0FB8A5B00FB8273
S11309807B8A013B7B827B8A002BE8D1BB8A013BBB
S1130990BB82BB8A002BD4D1FB8A18461C37BD46C8
S11309A05DF8047B704780B400AF00BFBD465DF8BE
S11309B0047B704780B588B000AFF8607A603B6014
S11309C00B46FB724FF6FF733B830023FB8200232D
S11309D0FB76A84B00221A60A74B00221A60A74B93
S11309E000221A60A64B00221A60A64B00221A802D
S11309F04FF480520021A44805F057FE55220021EF
S1130A00A24805F052FEFB7A012B0CD1F868FFF7DF
S1130A106BFF40F2054200219D4805F046FE43214C
S1130A20F868FFF749FF0121F868FFF771FF002319
S1130A307B7507F115031946F868FFF7F1FE7B7D16
S1130A40012B78D18521F868FFF762FF8422904951
S1130A50F868FFF7FBFE80218E48FFF765FF034629
S1130A60FB828B4B93F882303B833B8B1B023B8393
S1130A70874B93F883309AB23B8B13443B83FA8AB7
S1130A803B8B9A424AD10223BB8311E0BB8B804A41
S1130A90D35C002B03D1BB8B0133BB830BE0BB8B3B
S1130AA0BA8B7B49895C794AD154BB8B0133BB83B4
S1130AB0BB8B832BEAD9704B00221A6018E0BB8BE6
S1130AC0734AD35C7B757B7D2F2B14D97B7D392BAB
S1130AD011D8694B1A6813469B0013445B001A46ED
S1130AE07B7D1344303B644A1360BB8B0133BB836F
S1130AF0BB8B832BE3D9FFF756FF604B1A683B6827
S1130B0013445F4A13605E4B1A685B4B1B681946BB
S1130B10104600F059FC0023FB7691E040F20542B8
S1130B2000215B4805F0C1FDF868FFF7DDFE1521E3
S1130B30F868FFF7C1FE7B7D022B7FF474AF40F2AF
S1130B400541F868FFF7E4FE40F204425049F868B2
S1130B50FFF77CFE4FF480614E48FFF7E5FE034645
S1130B60FB824B4B93F802343B833B8B1B023B834E
S1130B70474B93F803349AB23B8B13443B83FA8A72
S1130B803B8B9A424ED10223BB8311E0BB8B404A7C
S1130B90D35C002B03D1BB8B0133BB830DE0BB8B38
S1130BA0BA8B3B49895C394AD154BB8B0133BB8333
S1130BB0BB8B40F203429342E8D92F4B00221A60C8
S1130BC018E0BB8B324AD35C7B757B7D2F2B16D907
S1130BD07B7D392B13D8284B1A6813469B0013448A
S1130BE05B001A467B7D1344303B234A1360BB8B66
S1130BF00133BB83BB8B40F203429342E1D9FFF73D
S1130C00D2FE1E4B1A683B6813441D4A13601C4BEA
S1130C101A68194B1B681946104600F0D5FB0023CF
S1130C20FB760DE040F205420021194805F03DFD38
S1130C30F868FFF759FE1521F868FFF73DFEF2E664
S1130C400D4B1B68B3F5001F00F20B8240F2054206
S1130C5000210F4805F029FD0621F868FFF72CFE56
S1130C604321F868FFF728FE064B00221A80002370
S1130C70FB77F1E17014002060140020641400205C
S1130C80681400206C1400200000002008140020C8
S1130C90001000200210002000237B750121F86859
S1130CA0FFF736FE07F115031946F868FFF7B8FD9C
S1130CB07B7D013B172B00F2CE8101A252F823F079
S1130CC0210D0000AB0E000057100000ED0F0000D6
S1130CD05710000057100000571000005710000074
S1130CE05710000057100000571000005710000064
S1130CF05710000057100000571000005710000054
S1130D005710000057100000571000005710000043
S1130D105710000057100000571000005110000039
S1130D208521F868FFF7F4FD8422A149F868FFF7EC
S1130D308DFD80219F48FFF7F7FD0346FB829C4B06
S1130D4093F882303B833B8B1B023B83984B93F895
S1130D5083309AB23B8B13443B83FA8A3B8B9A428F
S1130D6040F095800023BB8315E0BA8B924B1B683F
S1130D701A44924B1B689A4211D2914B1B881A4613
S1130D80BB8B1344BA8B02328949895C8D4AD15496
S1130D90BB8B0133BB83BB8B7F2BE6D900E000BF49
S1130DA0874B1A88BB8B13449AB2854B1A80BA8B33
S1130DB0814B1B681344804A136040F205420021B2
S1130DC07B4805F072FC7C4B1A687C4B1B689A428A
S1130DD02DD1794B1A687C4B1B689A421CD9764BEF
S1130DE01A68794B1B68D31AB3F5805F14D8774B14
S1130DF01B684FF480521946724800F01DFB6E4B7D
S1130E001B68714A1360704B1A683B6813446F4A3D
S1130E1013606B4B00221A800621F868FFF74CFD23
S1130E20FB7E022B40F018810123FB7714E1624B17
S1130E301A68654B1B689A421ED95F4B1A68624B4D
S1130E401B68D31AB3F5805F16D1604B1B684FF44F
S1130E50805219465B4800F0EFFA5B4B1B6803F5C0
S1130E608053594A1360584B1A683B681344574AD5
S1130E701360534B00221A8040F2054200214C4873
S1130E8005F013FC0621F868FFF716FDE4E040F2D4
S1130E9005420021464805F008FCF868FFF724FDE8
S1130EA01521F868FFF708FDD6E040F20541F8681F
S1130EB0FFF72EFD40F204423D49F868FFF7C6FCF7
S1130EC04FF480613B48FFF72FFD0346FB82384B0C
S1130ED093F802343B833B8B1B023B83344B93F8E4
S1130EE003349AB23B8B13443B83FA8A3B8B9A427A
S1130EF06ED10023BB8315E0BA8B2F4B1B681A44B9
S1130F002E4B1B689A4212D22D4B1B881A46BB8B60
S1130F101344BA8B02322649895C2A4AD154BB8BCA
S1130F200133BB83BB8BB3F5806FE5D300E000BF17
S1130F30234B1A88BB8B13449AB2214B1A80BA8B69
S1130F401D4B1B6813441C4A13601B4B1A681E4B31
S1130F501B689A421ED9184B1A681B4B1B68D31A7C
S1130F60B3F5805F16D1194B1B684FF480521946B4
S1130F70144800F061FA144B1B6803F58053124ABD
S1130F801360114B1A683B681344104A13600C4BEE
S1130F9000221A8040F205420021054805F085FB35
S1130FA0F868FFF7A1FC0621F868FFF785FC53E019
S1130FB00010002002100020701400206014002093
S1130FC06C14002000000020641400206814002029
S1130FD040F205420021254805F067FBF868FFF759
S1130FE083FC1521F868FFF767FC35E0204B1A688D
S1130FF0204B1B689A422FD1FB7E002B10D1FB7E25
S11310000133FB7640F205420021184805F04DFB00
S1131010F868FFF769FC1521F868FFF74DFC1BE041
S1131020FB7E012B18D1FB7E0133FB7640F2054297
S113103000210E4805F039FBF868FFF755FC06213E
S1131040F868FFF739FC4321F868FFF735FC03E043
S11310500123FB7700E000BFFB7F002B3FF41CAEB5
S113106000E000BF2037BD4680BD00BF0010002057
S1131070701400206014002080B586B000AF786042
S11310804FF0E0230D4AC3F8082D7B681B687B6191
S11310907B6804331B683B613B69FB607B69BB6015
S11310A0BB6883F308883B69B3F1FF3F02D072B693
S11310B0FB68984700BF1837BD4680BD0080FF1FFE
S11310C080B582B000AF414B1B6843211846FFF73F
S11310D0F3FB3F4B00221A603D4B1B68322B00D8B8
S11310E0FAE700BF0120FFF7CEFB0346842B09D9A2
S11310F0364B01221A60374B01221A60322002F06B
S113110073FF42E0314B1B681846FFF7BCFB0346F4
S1131110FB80FB88842B06D92E4B01221A603220D7
S113112002F062FF31E02B4B1B68002B1BD12A4BD2
S11311301A68274B1B689A4215D0254B1B68264A10
S11311401360234B1A68254BA3FB02131B0932219E
S113115001FB03F3D31A002B05D11C4B1B6843215D
S11311601846FFF7A9FB1B4B1B68002BCAD1184B71
S11311701B68632BC6D9322002F036FF134B1B6861
S11311801749184600F0ECFC1DE0104B1868154B8D
S11311901B6800220021FFF70DFC0D4B00221A6092
S11311A0322002F015FF0A4B1B68632B00D8FAE7C4
S11311B000BF322002F018FF044B1B680A4918468E
S11311C000F0CEFC00BF0837BD4680BDE886FF1F97
S11311D00084FF1FF04E0020EC86FF1F1F85EB519B
S11311E0F86E0000E486FF1F386F000080B586B0FB
S11311F000AF4FF4BE237B600023FB8209E0FB8A2F
S1131200FA8A79680A441178344AD154FB8A013342
S1131210FB82FB8A0F2BF2D94FF4C0237B60304B47
S113122000221A602D4B1B682E4A934251D12B4B3E
S11312301B7B012B4DD100233B612CE00023FB6081
S11312400EE0274B1A68FB6813447A681344197834
S1131250254AFB6813440A461A70FB680133FB6095
S1131260FB68B3F5805FECD31D4B1B6803F50033BB
S11312701E4A13601D4B1B684FF4805219461A48CE
S113128000F0DAF8164B1B6803F58053144A136018
S11312903B6901333B613B691F2BCFD94FF4BE231C
S11312A07B6000237B8106E07B890F4AFF21D154B8
S11312B07B8901337B817B89B3F5805FF4D34FF461
S11312C080524FF4BE21084800F0B6F800BF00BFBA
S11312D000BF00BF1837BD4680BD00BFE04E0020F0
S11312E0D84E002055AA5AA5F84E0020F44E0020EE
S11312F080B582B000AFFFF779FFFFF7E1FE02F09F
S11313008FFE0A4B1B681846FFF7B6FE02F07AFE02
S1131310074B1B687B60074B1B687A6806491846B5
S113132000F01EFC00BF0837BD4680BDE486FF1FE9
S113133024700000E886FF1F786F000080B400AFBF
S1131340064A064B5B78DBB203F07F03DBB25370D3
S113135000BFBD465DF8047B704700BF000002403B
S113136080B500AF134A134BD3F8003443F0300375
S1131370C2F800340F4A0F4BD3F8043443F030035F
S1131380C2F804340C4B4FF0FF329A6100220B492F
S1131390122002F0FDFD122002F01AFE02F032FECD
S11313A00549074802F03AFC03461A46054B1A80E1
S11313B000BF80BD00100040741400203D130000E5
S11313C0BC6F00009414002080B584B000AF786036
S11313D039603B681B0BFB603B68C3F30B03002BBA
S11313E002D0FB680133FB60104B114A9A61FB6821
S11313F01B031A4679680D4802F076FC03461A4628
S11314000C4B1A80094B4FF0FF329A613B681B0961
S11314109AB201237968054802F0B2FC03461A46E1
S1131420044B1A8000BF1037BD4680BD74140020E1
S11314305987FF1F9414002080B586B002AFF8606E
S1131440B9601346FB80322002F0CEFD174B184AD8
S11314509A614FF48052B968144802F045FC03467F
S11314601A46144B1A80114B4FF0FF329A61FA88D6
S1131470FB68B9680D4802F0B9FC03461A460D4BE7
S11314801A80FA88012301930B4B0093FB68B96817
S1131490064802F007FD03461A46064B1A8032201E
S11314A002F096FD00BF1037BD4680BD74140020C5
S11314B05987FF1F941400209014002080B582B037
S11314C002AF08230093144B144A1549154802F03F
S11314D0E9F91549154802F095F91549154802F03E
S11314E091F91549154802F08DF91549154802F08E
S11314F089F91549154802F085F91549154802F08E
S113150081F91549154802F07DF91549154802F08D
S113151079F900BFBD4680BDD46F0000F46F0000B0
S1131520D06F0000884D0020CC84FF1F084D0020A0
S1131530DC84FF1F184D0020EC84FF1F284D002081
S1131540FC84FF1F384D00200C85FF1F484D0020F0
S11315501C85FF1F584D00202C85FF1F684D00205F
S11315603C85FF1F784D002080B500AF0023104A52
S11315700121104801F064FF0121002001F06EFFF9
S113158000230D4A01210D4804F0F6FF012101203A
S113159005F008F80A49052004F0BDFBFFF78EFFAB
S11315A000F0A4FB00F00EF8FFF7DAFE00BF80BDE8
S11315B0044D00208084FF1F644E00202486FF1FFA
S11315C0AC85FF1F80B500AF1C49002003F064F90F
S11315D01B4A0021002003F013FA1A4A01210020BB
S11315E003F00EFA184A0221002003F009FA174A00
S11315F00321002003F004FA00221549302002F0F0
S1131600C7FC00221349312002F0C2FC0022124917
S1131610322002F0BDFC00221049332002F0B8FC55
S11316200421002003F08EF90221322002F000FD93
S1131630322002F0CDFC00BF80BD00BF147000005A
S11316404C85FF1F6485FF1F7C85FF1F9485FF1F4A
S11316508987FF1FA987FF1FC987FF1FE987FF1F0E
S113166080B487B000AF786039607B681B89BB8227
S11316707B685B691B78FB747B681B69FB607B6818
S11316805B68BB60BB681B88FB82FB8AFA681344F7
S1131690FA7C1A70FB8A0133FB82FA8ABB8A9A426B
S11316A001D10023FB82BB68FA8A1A803B680122BD
S11316B01A607B685B6918461C37BD465DF8047B7D
S11316C07047000080B485B000AFF8600B467A60C4
S11316D0FB72FB7A022B02D1044B01221A7000BF69
S11316E01437BD465DF8047B704700BF0484FF1FB8
S11316F080B588B000AFF8600B467A60FB72FB6877
S1131700BB617B687B61BB6993F82830002B72D185
S1131710FB7A042B3BD1BB69DB683B613B69002B43
S113172004D03B69C3F50063FB6102E04FF400633E
S1131730FB613A4B1B889BB21A46FB691344B3F511
S1131740006F14D2354B1B889BB21A46344B13449A
S1131750FA693449184604F09DFFFB699AB22F4B8D
S11317601B889BB213449AB22C4B1A8002E02E4B76
S113177001221A704FF4006200212A4804F095FFF8
S11317804FF400622749002003F082FE41E0FB7A17
S1131790002B3ED14FF40063FB61204B1B889BB2AE
S11317A01A46FB691344B3F5006F14D21B4B1B8814
S11317B09BB21A461A4B1344FA691A49184604F0A4
S11317C069FFFB699AB2154B1B889BB213449AB20A
S11317D0124B1A8002E0144B01221A704FF400627B
S11317E00021104804F061FF4FF400620D4900200D
S11317F003F052FF0DE0BB6993F82830012B08D1A8
S1131800BB690C3319467869FFF72AFF0246BB69A6
S11318105A6000BF2037BD4680BD00BFA62C002003
S1131820A4240020A41C0020A42C002080B485B093
S113183000AFF8600B467A60FB72FB7A022B02D190
S1131840044B01221A7000BF1437BD465DF8047BB7
S1131850704700BF0584FF1F80B588B000AFF860F3
S11318600B467A60FB72FB68BB617B687B61BB697A
S113187093F82830002B72D1FB7A042B3BD1BB693F
S1131880DB683B613B69002B04D03B69C3F5006313
S1131890FB6102E04FF40063FB613A4B1B889BB28F
S11318A01A46FB691344B3F5006F14D2354B1B88F9
S11318B09BB21A46344B1344FA693449184604F06F
S11318C0E9FEFB699AB22F4B1B889BB213449AB270
S11318D02C4B1A8002E02E4B01221A704FF4006246
S11318E000212A4804F0E1FE4FF400622749012058
S11318F003F0CEFD41E0FB7A002B3ED14FF40063B0
S1131900FB61204B1B889BB21A46FB691344B3F559
S1131910006F14D21B4B1B889BB21A461A4B1344FC
S1131920FA691A49184604F0B5FEFB699AB2154BD8
S11319301B889BB213449AB2124B1A8002E0144BD8
S113194001221A704FF400620021104804F0ADFE29
S11319504FF400620D49012003F09EFE0DE0BB69C7
S113196093F82830012B08D1BB690C3319467869E8
S1131970FFF776FE0246BB695A6000BF2037BD46BA
S113198080BD00BFC63C0020C4340020C42C00200D
S1131990C43C002080B485B000AFF8600B467A6088
S11319A0FB72FB7A022B02D1044B01221A7000BF96
S11319B01437BD465DF8047B704700BF0584FF1FE4
S11319C080B588B000AFF8600B467A60FB72FB68A4
S11319D0BB617B687B61BB6993F82830002B72D1B3
S11319E0FB7A042B3BD1BB69DB683B613B69002B71
S11319F004D03B69C3F50063FB6102E04FF400636C
S1131A00FB613A4B1B889BB21A46FB691344B3F53E
S1131A10006F14D2354B1B889BB21A46344B1344C7
S1131A20FA693449184604F035FEFB699AB22F4B23
S1131A301B889BB213449AB22C4B1A8002E02E4BA3
S1131A4001221A704FF4006200212A4804F02DFE8E
S1131A504FF400622749022003F01AFD41E0FB7AAB
S1131A60002B3ED14FF40063FB61204B1B889BB2DB
S1131A701A46FB691344B3F5006F14D21B4B1B8841
S1131A809BB21A461A4B1344FA691A49184604F0D1
S1131A9001FEFB699AB2154B1B889BB213449AB2A0
S1131AA0124B1A8002E0144B01221A704FF40062A8
S1131AB00021104804F0F9FD4FF400620D490220A2
S1131AC003F0EAFD0DE0BB6993F82830012B08D13F
S1131AD0BB690C3319467869FFF7C2FD0246BB693E
S1131AE05A6000BF2037BD4680BD00BFE64C0020D1
S1131AF0E4440020E43C0020E44C002080B487B09F
S1131B0000AF78600D4A07F1080307CA83E80700AD
S1131B107B689B0007F11802134453F8103C7B6167
S1131B207B695B6800221A807B691B6800221A802B
S1131B3000BF1C37BD465DF8047B7047A46F0000EE
S1131B4080B582B000AF78600B46FB70FB1C0122AD
S1131B501946786803F05AFC00BF0837BD4680BDBB
S1131B600EB480B585B000AF78600023FB6007F148
S1131B702003BB60BA68F9690E4804F0B7FD034658
S1131B80FB60FB68B3F5006F00D9FEE77B68012BAF
S1131B9002D07B68022B04D1FA680649786803F006
S1131BA035FCFB6818461437BD46BDE8804003B0D9
S1131BB0704700BFA414002080B489B000AF7860DF
S1131BC03960194A07F1100307CA83E807007B68E4
S1131BD09B0007F12002134453F8103CFB61FB699E
S1131BE05B681B88FB81FB691B681B88BB81FB89C5
S1131BF09AB2BB899BB29A42F1D9FB691A69BB8933
S1131C009BB2591C89B2B98113441A783B681A7083
S1131C10FB691B68BA8992B21A8000BF00BF2437DF
S1131C20BD465DF8047B7047A46F000080B58AB0A0
S1131C3000AFF860B9601346FB801B4A07F110033C
S1131C4007CA83E80700FB689B0007F128021344D6
S1131C5053F8183C7B627B6A5B681B887B847B6AD5
S1131C601B681B883B847A8C3B8C9A42F3D97A8C10
S1131C703B8CD31AFB83FA8BFB889A4200BF7B6AA6
S1131C801A693B8C1344FA881946B86804F002FDBB
S1131C907B6A1B68398CFA880A4492B21A8000BFA6
S1131CA02837BD4680BD00BFA46F000080B489B052
S1131CB000AF78600C4A07F10C0307CA83E80700F9
S1131CC07B689B0007F12002134453F8143CFB612A
S1131CD0FB695B681B887B837B8B18462437BD4676
S1131CE05DF8047B704700BFA46F000080B500AFAF
S1131CF0514A5249002003F055FC514B4FF4006205
S1131D001A814F4B4F4A5A604D4B4F4A1A604C4B05
S1131D104E4ADA604A4B4E4A5A61494B4D4A1A615F
S1131D20474A4D49002003F05DFB00224B49002047
S1131D3003F062FB404BDB79002B06D14FF40062C9
S1131D404349002003F0A4FB08E03B4BDB79012B63
S1131D5004D101223E49002003F09AFB404A414944
S1131D60012003F01FFC404B4FF400621A813E4BEC
S1131D703E4A5A603C4B3E4A1A603B4B3D4ADA604D
S1131D80394B3D4A5A61384B3C4A1A61364A3C4900
S1131D90012003F027FB00223A49012003F02CFB29
S1131DA02F4BDB79002B06D14FF40062324901201E
S1131DB003F06EFB08E02A4BDB79012B04D10122EE
S1131DC02D49012003F064FB2F4A3049022003F01F
S1131DD0E9FB2F4B4FF400621A812D4B2D4A5A60B8
S1131DE02B4B2D4A1A602A4B2C4ADA60284B2C4A7A
S1131DF05A61274B2B4A1A61254A2B49022003F0CA
S1131E00F1FA00222949022003F0F6FA1E4BDB798D
S1131E10002B06D14FF400622149022003F038FB65
S1131E2008E0194BDB79012B04D101221C49022063
S1131E3003F02EFB00BF80BD18700000C84D0020C9
S1131E40AC2C0020A62C0020A82C0020A42C0020C0
S1131E50A41C0020A4240020F1160000C5160000D4
S1131E6024700000FC4D0020CC3C0020C63C002027
S1131E70C83C0020C43C0020C42C0020C4340020F2
S1131E80591800002D18000030700000304E00205A
S1131E90EC4C0020E64C0020E84C0020E44C0020F0
S1131EA0E43C0020E4440020C1190000951900001E
S1131EB04FF0E023D3F8882D42F47002C3F8882D44
S1131EC0D3F8342F22F08042C3F8342F054B064A4E
S1131ED05A605A6842F220121A604FF6FF729A60F2
S1131EE0704700BF0020054020C528D9264B274A4B
S1131EF09A4208D013462448254A13F8011B02F8D5
S1131F00011B9842F9D1234B234A9A4208D0134625
S1131F102048224A13F8011B02F8011B8342F9D11D
S1131F201F4B204A9A4206D0134600211C4A03F84C
S1131F30011B9342FBD11C4B1C4A9A4208D0134606
S1131F4019481B4A13F8011B02F8011B8342F9D1FB
S1131F50184B194A9A4212D010B4184CA40808D04D
S1131F601946002351F8040B42F8040B0133A34231
S1131F70F8D1134B104A1A605DF8044B7047104BAC
S1131F800C4A1A60704700BF04760000B07200006B
S1131F900084FF1FF4760000047600005887FF1FBA
S1131FA0085F002000000020F4760000F4760000B2
S1131FB000000020000000000080FF1F000400005B
S1131FC008ED00E0074B5B69DBB2042B06D0802BE5
S1131FD006D0012B0CBF012004207047022070475B
S1131FE00320704700E00740044BD3F8003113F09E
S1131FF0807F1ABF024B18680020704700400640DB
S1132000884E002010B584B00B4600293BD0444ACA
S1132010D2F8002112F0007F7DD1414AD2F800119C
S113202021F40001C2F800114FF08061C2F80011E0
S113203000213C4A1160002870D05A7A120202F43E
S1132040E062197A01F007010A433548C0F8042117
S1132050DA79120102F030029979C90001F008011D
S11320600A435979890001F004010A43C0F80821A0
S11320701A79012A29D0E2B1022A32D01A68294BEE
S11320801A60294C3BE000238DF804308DF80C30A5
S113209001228DF808208DF809208DF805208DF88F
S11320A0063002238DF8073004AB204A43F8102D84
S11320B0ADE71A7B002A14BF4FF40002002242F05D
S11320C001021749C1F80021D8E71A7B002A14BF7E
S11320D04FF40002002242F001121149C1F800211C
S11320E0CCE71A7B002A14BF4FF403024FF44032AA
S11320F042F001020A49C1F80021BFE7013CFFF7A1
S113210073FF18B9002CF9D1032005E0002C14BF8B
S11321100020032000E0022004B010BD0020FBE7F3
S113212000400640884E002088E7300000127A0004
S1132130084BD3F8003213F0807F09D0054BD3F855
S1132140083203F00103002B034808BF0020704746
S1132150002070470040064000127A0010B582B09B
S11321600B46002938D02D4AD2F8002212F0007F05
S11321704FD12A4AD2F8001221F40001C2F8001209
S11321800021C2F80012002846D09A78120202F404
S1132190E062597801F007010A432049C1F804229A
S11321A01A7802F00102C1F8082259799A791B7948
S11321B0002B14BF03230123002914BF0421002191
S11321C00B43002A14BF4FF4000200221343134AA6
S11321D0C2F80032642410E000238DF80430012298
S11321E08DF805208DF806308DF801208DF8022039
S11321F002AB03F8082DB6E7013CFFF799FF18B9C5
S1132200002CF9D1032005E0002C14BF002003208A
S113221000E0022002B010BD0020FBE700400640B1
S1132220054BD3F8003313F0807F1DBF024BD3F866
S1132230083302480020704700400640006CDC026E
S113224010B582B00B46002932D0294AD2F80023B7
S113225012F0007F47D1264AD2F8001321F400017E
S1132260C2F800134FF08061C2F8001300283DD07B
S11322709A78120202F4E062597801F007010A43E5
S11322801B49C1F804231A7802F00302C1F8082399
S11322909A795B79002B14BF01230923002A14BF08
S11322A04FF4000200221343C1F8003364240EE00B
S11322B001238DF8053000228DF806208DF80130B9
S11322C08DF8023002AB03F8082DBEE7013CFFF79E
S11322D0A7FF18B9002CF9D1032005E0002C14BF86
S11322E00020032000E0022002B010BD0020FBE724
S11322F00040064008B50F4BD3F8003613F0807F3A
S113230002D10023184608BDFFF76EFE03460028DD
S1132310F8D00849D1F80826C2F302220132B0FBF2
S1132320F2F3D1F80826C2F30442103203FB02F39D
S11323305B08E7E70040064010B584B00C4699B14D
S11323403D4BD3F8003613F0007F72D13A4BD3F8EB
S1132350002622F40002C3F800264FF08062C3F87E
S11323600026A0B9002065E000238DF804308DF824
S11323700B3001228DF808208DF809208DF80530E6
S113238007228DF806208DF8073001ACD8E7FFF757
S11323902BFE63791B0203F4E063227902F0070247
S11323A013432549C1F8043663781B0203F4E06340
S11323B0A278120402F4F8121343C1F80836237801
S11323C0012B16D04BB1022B1FD04FF47A74FFF7B8
S11323D091FF48BB34B3013CF9E7E379002B14BF08
S11323E04FF40003002343F00103134AC2F80036FC
S11323F0EBE7E379002B14BF4FF40003002343F011
S113240001130D4AC2F80036DFE7E379002B14BF4D
S11324104FF403034FF4403343F00103064AC2F878
S11324200036D2E7032005E0002C14BF002003206F
S113243000E0022004B010BD004006402DE9F04148
S113244080460D468C7801344E7806FB04460F789E
S113245007FB0447CB78013B052B1CD8DFE803F0CE
S11324600312151B1B18FFF7BFFD0009B8F1020F7B
S11324704AD0B8F1030F7BD0B8F1010F0DD0002082
S1132480BDE8F081FFF754FEEFE7FFF7C9FEECE784
S1132490FFF730FFE9E70020E7E7EA7802EB4201C3
S11324A05B4B53F821301B0904FB03F4A04200F2F8
S11324B093800B46564901EB83035B681B0906FBBB
S11324C003F6B04200F28B8002EB420301EB83037C
S11324D09B681B0907FB03F7B84200F28380AB78C3
S11324E01B0403F47023120602F0706213432A786B
S11324F002F00F0213436A781201D2B21343454A21
S113250053610020BDE8F081EA7802EB4201424BBE
S113251053F821301B0904FB03F4A04265D80B4691
S11325203D4901EB83035B681B0906FB03F6B042DC
S11325305ED802EB420301EB83039B681B0907FB94
S113254003F7B84257D8AB781B0403F47023120680
S113255002F0706213432A7802F00F0213436A7880
S11325601201D2B213432B4A93610020BDE8F081DB
S1132570EB7803EB4301294A52F82120120904FBAA
S113258002F4A0423AD80A46244901EB8202526876
S1132590120906FB02F6B04233D803EB430201EB07
S11325A082029268120907FB02F7B8422CD8AA7873
S11325B0120402F470221B0603F0706313432A789A
S11325C002F00F0213436A781201D2B21343114A84
S11325D0D3610020BDE8F0810120BDE8F081012035
S11325E0BDE8F0810120BDE8F0810120BDE8F08163
S11325F00120BDE8F0810120BDE8F0810120BDE8A3
S1132600F0810120BDE8F0810120BDE8F08100BF28
S1132610307100000040064084710000DC7000004E
S113262038B50546FFF7CEFC2946FFF707FF0446F9
S113263058B9E8780A220849013A0B69C3F30363DD
S1132640984204D0002AF7D10324204638BD002A3A
S113265008BF0324F9E700BF0040064010B5044654
S11326601B4B1B69C3F30363013B052B1DD8DFE838
S113267003F00313161C1C19FFF7B6FC144B1B695B
S1132680C3F303430133B0FBF3F0012C0FD0ECB1DF
S1132690022C14D0002010BDFFF74AFDEEE7FFF72F
S11326A0BFFDEBE7FFF726FEE8E70020E6E7084B6F
S11326B01B69C3F303130133B0FBF3F010BD044BE8
S11326C01B6903F00F030133B0FBF3F010BD00BF2F
S11326D00040064008B50F4B1B6AC3F30363062B87
S11326E015D8DFE803F004080B0E141411000220BF
S11326F0FFF7B4FF08BDFFF777FC08BDFFF718FD2F
S113270008BDFFF78DFD08BDFFF7F4FD08BD0020EF
S113271008BD00BF0040064008B541B1012931D0D1
S11327200020024610B1431E22FA03F008BD04380B
S1132730032852D8DFE800F00B02141DFFF770FDE8
S11327400246294BD3F8040300F00700EAE7FFF739
S1132750EFFC0246244BD3F8040200F00700E1E743
S1132760FFF742FC0246204BD3F8040100F00700B7
S1132770D8E7FFF7BFFD02461B4BD3F8040600F071
S11327800700CFE7043803282AD8DFE800F00B025B
S1132790141DFFF745FD0246134BD3F80403C0F3A1
S11327A00220BFE7FFF7C4FC02460F4BD3F8040234
S11327B0C0F30220B6E7FFF717FC02460A4BD3F832
S11327C00401C0F30220ADE7FFF794FD0246064B77
S11327D0D3F80406C0F30220A4E700200246A1E7D0
S11327E0002002469EE700BF0040064008B5114B9A
S11327F01B69C3F30113032B19D8DFE803F00207A5
S1132800101300210620FFF787FF08BD094B186944
S113281000F00200002818BF4FF4FA4008BD064B30
S1132820186808BD00210520FFF776FF08BD0020C9
S113283008BD00BF00800440684E002038B51C4B22
S113284033F810309B0003F1804303F5CA231D685D
S1132850C5F3C0051C6804F00704AC4225D318680E
S1132860C0F3807010B31B68C3F30263013B052BF4
S113287019D8DFE803F0030C101818140620FFF72A
S11328804BFF0134B0FBF4F005FB000038BD04201D
S1132890FFF742FFF5E70520FFF73EFFF1E70720CA
S11328A0FFF73AFFEDE70020EBE7002038BD00BF5B
S11328B03C700000114B1B69C3F38103022B07D04A
S11328C0032B0ED0002B0CBF4FF4FA3000207047BE
S11328D00A4B186900F00200002818BF4FF4FA40B0
S11328E07047064B186910F0020006D0186900F012
S11328F00100002818BF4FF47A707047008004402C
S113290008B5244B5B6813F4006F40D0214B5B681F
S1132910C3F303130E2B09D8DFE803F00A080D08EC
S11329201208171C20252F0829082C00002026E057
S1132930FFF7D0FE23E001210620FFF7EDFE1EE0A5
S113294001210420FFF7E8FE19E001210520FFF72B
S1132950E3FE14E00020FFF781FE10E001210720D0
S1132960FFF7DAFE0BE00120FFF778FE07E0FFF740
S1132970A1FF04E0FFF73AFF01E04FF4FA30054B02
S11329805B68C3F302230133B0FBF3F008BD0020FE
S113299008BD00BF00800440F0B5A1B028B30446D0
S11329A00646002800F0FF80644B1B69C3F30363F1
S11329B0032B00F0C980FFF733FC002800F0B4803B
S11329C003238DF8073000228DF8062001228DF8AC
S11329D0052020A800F87C3DFFF722FE05460028CC
S11329E000F0B280284621B0F0BD01238DF80B30F1
S11329F000228DF80C208DF80D308DF80E208DF806
S1132A0008308DF809308DF80A308DF816308DF8BD
S1132A1014308DF815208DF80F208DF810308DF8B6
S1132A2011308DF838300D928DF8253044490691D7
S1132A308DF81C208DF824208DF81D308DF81E2073
S1132A4002208DF81F008DF820308DF821308DF88C
S1132A5030308DF828208DF82F208DF829200C2176
S1132A608DF82A108DF82B208DF82C308DF82D3010
S1132A708DF83D3003218DF83C108DF84B308DF8E6
S1132A8041108DF840208DF83F308DF83E308DF8A0
S1132A9045008DF844308DF843208DF8421006200F
S1132AA08DF849008DF848208DF847308DF8461090
S1132AB024491E9120211D918DF84C308DF84D2014
S1132AC08DF84E208DF84F208DF850308DF854300D
S1132AD08DF853308DF852208DF851208DF86830E0
S1132AE08DF869308DF86A308DF86B308DF86C3064
S1132AF08DF86D308DF873308DF858301792189228
S1132B0019928DF86E308DF86F308DF870208DF835
S1132B1071208DF872208DF87C308DF87D308DF821
S1132B207E2002AE34463FE700210120FFF788FBF8
S1132B30054600287FF456AF42E700BF0040064038
S1132B4000127A002C86FF1F3146E078FFF706FB5F
S1132B500546002800F02381FFF734FA022800F02C
S1132B605881032800F05881012800F03281002D9B
S1132B707FF438AF94F8303013B1E26AA84B1A608E
S1132B8094F8353053B1A7490A6A22F0706294F878
S1132B9034301B0603F0706313430B6294F8433024
S1132BA0002B40F0A68114F16C0F35D0236F002B5D
S1132BB032D0E36E83B300219B489C4D01EB81022C
S1132BC0236F9B5C30F813309B0003F1804303F5C3
S1132BD0CA231E6826F080461E60236F9F189E5CE1
S1132BE0BB781B0603F0E063FA78D20002F0080217
S1132BF013433A7902F0070213437A78002A14BF88
S1132C004FF080420022134330F8162045F822305A
S1132C100131E36E9942D1D394F84430C3B194F8AE
S1132C20463094F847208249496821F47F6194F83A
S1132C304500002814BF4FF4006000201B01DBB2E4
S1132C40120202F4E06213430B430343784A5360D5
S1132C5094F84830DBB194F84A3094F84920744928
S1132C60096921F03F0194F84C00084394F84B1093
S1132C70002914BF022100219B0003F00C0303432D
S1132C80120102F0300213430B43694A136194F8B2
S1132C906030002B37D0664B196C21F0010194F899
S1132CA061200A431A641B6C23F0020394F8622027
S1132CB0002A14BF0222002213435D4A1364136CDA
S1132CC023F0040394F86320002A14BF0422002292
S1132CD01343574A1364136C23F0080394F86420D5
S1132CE0002A14BF082200221343514A1364136CB0
S1132CF023F0100394F86520002A14BF1022002248
S1132D0013434B4A136494F8503033B1494B626D0A
S1132D101A60A26D5A60E26D9A6094F86630EBB165
S1132D20434A936E00209066516821F4805194F8D0
S1132D3068301B0303F480530B435360906694F88C
S1132D4067305BB194F869305B0003F00E0394F8CC
S1132D506A2042F080521343354A936694F87430E3
S1132D60002B00F0E28034498B7803F07F0394F861
S1132D70752082F0010243EAC213DBB28B7094F92E
S1132D807630002BBCBF20335BB22B490A7903F0A9
S1132D901F0302F0E00213430B71002522E604F145
S1132DA01001607FFFF72EF9054600287FF4D4AEAA
S1132DB004F1200194F82800FFF7BEFA0546FFF756
S1132DC001F9022825D0032826D0012801D00026A5
S1132DD001E004F13606002D7FF4C9AEF378032B2D
S1132DE02CD08DF80730B3788DF8063073788DF8D1
S1132DF00530337820A800F87C3DFFF711FC054628
S1132E0000287FF4B4AEE11DA07BFFF719FA054654
S1132E10ADE604F13A06DEE704F13E06DBE700BF67
S1132E20684E0020004006403C7000000050064000
S1132E30008004406C4E002000D0074094F82830F5
S1132E400BBB637F93BBE378002B42D10125002D9C
S1132E507FF48DAEE11DA07BFFF7F2F90546002853
S1132E607FF485AEF3788DF80730B3788DF80630AB
S1132E7073788DF80530337820A800F87C3DFFF78F
S1132E80CFFB054673E606238DF8073002238DF841
S1132E90063001238DF8053020A800F87C3DFFF7AB
S1132EA0BFFB0546637F7BB10128D0D101238DF898
S1132EB0073000228DF806208DF8053020A800F890
S1132EC07C3DFFF7ADFB0546E378002BBFD0012D19
S1132ED0BDD102238DF8073000238DF806308DF81C
S1132EE0053020A8012300F87C3DFFF799FB054637
S1132EF0ADE704F136010120FFF7A0FA05460028EA
S1132F007FF470AD04F13A010220FFF797FA054609
S1132F1000287FF467AD04F13E010320FFF78EFA29
S1132F20054600287FF45EAD3DE600255AE500BF66
S1132F3070B504460D46112807D9232840F2858030
S1132F404D2840F25681042070BD11287AD8DFE85C
S1132F5000F00913191F24292E33383C41484F56D9
S1132F605D646B720020FFF779FB03460020002D9F
S1132F7000F0B2812B6070BD0120FFF76FFB0346A8
S1132F800020F4E70220FFF769FB03460020EEE788
S1132F90FFF7B6FC03460020E9E7FFF7C9F803464C
S1132FA00020E4E7FFF73CF903460020DFE7FFF7E2
S1132FB01BF803460020DAE7FFF79CF903460020DC
S1132FC0D5E7AC4B1B680020D1E7FFF783FB034632
S1132FD00020CCE700210420FFF79EFB03460020DD
S1132FE0C5E701210420FFF797FB03460020BEE755
S1132FF000210520FFF790FB03460020B7E70121DD
S11330000520FFF789FB03460020B0E700210620D6
S1133010FFF782FB03460020A9E701210620FFF702
S11330207BFB03460020A2E700210720FFF774FB87
S1133030034600209BE701210720FFF76DFB0346B1
S1133040002094E70023042091E7A0F115040E2C3E
S113305000F29E80DFE804F00814202B353E434F35
S11330605F6A727B848C9400834BDB68C3F30163D7
S1133070022B00F29080814A52F82330002024E091
S11330807D4BDB68C3F38163022B00F287807B4AAC
S113309052F82330002018E0774BDB68C3F3017348
S11330A0022B7ED8754A52F8233000200DE0724B73
S11330B0DB689B0F022B77D8704A52F8233000202C
S11330C003E0FFF71DFC03460020002D00F00481FF
S11330D02B6070BDFFF78AFB03460020F5E7684BC1
S11330E09B78DB0902D000231846EEE7FFF7E2FBEA
S11330F003460020E9E7624B9B78DB0957D15E4B1E
S11331001B6913F0020355D05B4B1B6913F00103D9
S113311052D10020D9E75A4B9B78DB0950D1564B4A
S11331201B6913F002034ED10020CEE7544B9B7869
S1133130DB094CD14FF4FA330020C6E74E4B1B6C2D
S1133140C3F30013002B45D14FF48070BDE74A4B05
S11331501B6CC3F3C003002B3FD14FF48070B4E762
S1133160454B1B6CC3F38003D3BB4FF48070ACE7B7
S1133170414B1B6CC3F34003ABBB4FF48070A4E71B
S11331803D4B1B6C13F0010330D14FF480709CE76E
S11331900023042099E70023184696E700231846E5
S11331A093E70023184690E7002318468DE7002391
S11331B018468AE7002088E74FF47A73002084E7F2
S11331C00023184681E74FF4FA4300207DE70023EB
S11331D018467AE70023184677E70023184674E771
S11331E00023184671E7002318466EE700231846AB
S11331F06BE7242805D804200023002D6CD02B6015
S113320070BDA0F13303DBB21A2B07D81D4A22FA92
S113321003F313F0010F18BF0420EDD11A4B33F858
S113322014201A4B53F8223013F0804F43D14FF43B
S11332308070E1E70120FFF711FA002846D100234E
S11332404FF48070D9E70020FFF708FA0028F6D081
S11332503CE00220FFF702FA0028F0D036E016F036
S1133260080F15D116F0100F1AD100234FF48070F7
S1133270C3E700BF684E0020008004406C4E00206D
S113328000D00740412100043C700000005006407B
S113329000212046FFF7D2FA034616F0100F04D09F
S11332A001212046FFF7CAFA0346002B14BF002071
S11332B04FF48070A1E7094B1E5D16F0200FB9D1C1
S11332C016F0400FBFD116F0800FC2D116F0180FC0
S11332D0C5D10023184690E770BD00BFD871000027
S11332E070B582B005460C46FEF76CFE06469DB1ED
S11332F02B68022B0ED0042B10D0012B0CBF012500
S113330004256CB12378043B032B4AD8DFE803F08F
S11333104B4345470225F4E70546F2E70325F0E76A
S1133320FEF77EFF58B103238DF8073000228DF895
S1133330062001228DF805208DF8043043E0FEF7C5
S1133340D9FF58B106238DF8073002238DF80630D3
S113335001238DF805308DF8043034E0FEF744FE87
S113336050B101238DF8073000228DF806208DF826
S113337005308DF8043026E0FEF7DAFE18B3022398
S11333808DF8073000238DF806308DF805300123C1
S11333908DF8043017E0032306E0012304E006233C
S11333A002E0FF2300E002238DF807300C4B628813
S11333B09A5C8DF80620A2889A5C8DF80520E28834
S11333C09B5C8DF80430B54205D001A92846FFF76F
S11333D035F802B070BD01A8FFF722F9F9E700BF84
S11333E028720000154B1B69C3F30363013B052BD3
S11333F020D8DFE803F00316191F1F1C06230370EF
S11334000E4A1369C3F30343013343801369C3F3BF
S1133410031301338380136903F00F030133C38063
S1133420704704230370EBE705230370E8E70723E1
S11334300370E5E704230370E2E700BF00400640A1
S113344010B4054C20602171A260237363730020C3
S11334505DF8044B704700BF784E0020F0B583B090
S113346007460E468DF804008DF8051000F0D8FDCF
S1133470334B1C7B5C7301238DF80630002C4AD03F
S113348000242F4D04E00134E4B22B7BA34242D943
S1133490AB6853F82430002BF5D01A79022AF2D005
S11334A01A68996801A890470028ECD06C73002E24
S11334B0E9D140F2031500238DF80630A400204E14
S11334C020E00134E4B23B7BA34212D9BB6853F839
S11334D02430002BF5D01A79012AF2D01A689968A1
S11334E001A890470028ECD07C73002EE9D14FF45A
S11334F0827500F087FD284603B0F0BD043C14F14A
S1133500040FF6D0B3681B59002BF7D01A689968DA
S113351001A89047F2E70A4D2B6853F82700FFF7FC
S11335203BFA6F7105460028C5D102238DF8063099
S1133530034B1B7B002BDCD00024014FC6E700BFEC
S1133540784E002008B5FFF7F3FC08BD29B14118F7
S1133550002300F8013B8142FBD1704710B4064BB5
S11335601B6853F82040616053F820309A600020B3
S11335705DF8044B704700BF8C4E002008B5084B23
S11335801B6853F8203000F00F00064A1077D077FC
S113359023B15A6812B1197B9868904708BD00BFDF
S11335A08C4E00200080004038B5054600F00F0422
S11335B000222146094800F000FA094B1B6853F821
S11335C0253053B1054A1477D477947701221A73BE
S11335D05A6812B1197B9868904738BD0080004042
S11335E08C4E00202DE9F04F87B09DF84070119D5E
S11335F00124BC405FFA84FCB5FBFCF60CFB1656B8
S1133600002E14BF4FF0010A4FF0000A03D05046B9
S113361007B0BDE8F08F059304920391804600F053
S11336200F06DFF800913146484600F0CBF9D9F88F
S1133630003043F08003C9F80030730103F1804285
S113364002F5004B02F51042049810604B4441F21D
S11336501002059898500197009700231A463146A6
S1133660484600F0E5F9039B032B12D8DFE803F08A
S1133670022D3D4C002241F204032BF8032064B2D6
S1133680A4B2730103F1804303F5004341F2140231
S11336909C52244C2A463146204600F0E1F901228E
S11336A03146204600F00AFA04EB461641F21C02A9
S11336B0B35A1BB243F002039BB2B3521A4B1B68BA
S11336C053F8283000221A73A1E764B2A4B241F27D
S11336D004032BF80340730103F1804303F5004313
S11336E0002141F214029952D3E764B2A4B241F228
S11336F004032BF80340730103F1804303F50043F3
S113370041F214029C52C4E7002241F204032BF854
S11337100320730103F1804303F5004341F21401D4
S11337205A52B6E7008000408C4E002070B582B03B
S11337300446079D01959DF818500095FFF752FF28
S1133740054610B1284602B070BD04F00F040F4EB8
S1133750089A2146304600F0B1F906EB441641F2CE
S11337601C03F35A23F008031B041B0C9DF82420AC
S1133770002A14BF082200221343640104F1804488
S113378004F5004441F21C02A352DBE70080004030
S113379008B5012200F00F01024800F00EF90020E4
S11337A008BD00BF0080004008B5002200F00F01F2
S11337B0024800F002F9002008BD00BF008000406C
S11337C010B40F4B1C5C04F07F041C541C5C01F00F
S11337D03F0104F0C004214319541B5C03F0BF03F0
S11337E0002A14BF402200221A43054B1A541A5CC3
S11337F042F080021A5400205DF8044B704700BF69
S1133800001002402DE9F04180460C464D7805F049
S11338100F061021FFF79AFE227BA1786078FFF74C
S1133820CFFF074631461D4800F0CCF817B13846A3
S1133830BDE8F0811A4B1B6843F8258053F8252016
S1133840157053F8253000221A73144D01223146A5
S1133850284600F0ADF82B6813F0040F11D123783B
S1133860FF2B0ED086F0030606F1804606F50046CF
S113387096F8002103F00F0302F0F002134386F8D8
S113388000316568A1686278054B1B6853F8220013
S1133890456053F822309960C9E700BF00800040BA
S11338A08C4E00202DE9F0420D4616469946069F9F
S11338B0244B18604021FFF749FE234C204600F0BA
S11338C0A6F8226822F004022B789B0003F004037C
S11338D013432360236823F010036A78002A14BF7B
S11338E01022002213432360102000F071FB174DB7
S11338F06C1E0F3514F9010F00F06AFBAC42F9D1CC
S1133900134800F020F9DEB1B9F1000F14D0AFB1C3
S1133910043EA9F1040900252C4659F8041F56F861
S1133920040FFFF76FFF002818BF05460134A742B4
S1133930F3D12846BDE8F0820025FAE70025F8E730
S11339400025F6E78C4E0020008000403C72000009
S11339500010024000F00F00400100F1804000F52B
S1133960004041F20C03C150704700F00F004001C9
S113397000F1804000F5004041F21003C15070474F
S113398008B50A4600F00F01014800F097F808BD99
S11339900080004008B500F00F01024800F0BDF8B7
S11339A008BD00BF00800040004870470080004010
S11339B00AB901767047417670470AB98176704733
S11339C0C176704700EB4111002341F208028B508D
S11339D001F58052136041F204028B5241F2060257
S11339E08B5241F20C028B5041F210028B5041F287
S11339F014028B5241F216028B5241F218028B5080
S1133A0041F21C028B5241F21E028B52704738B5B0
S1133A100546036823F4403323F0C60303600024FF
S1133A20E1B22846FFF7CEFF0134102CF8D138BD9F
S1133A3010B4DB00DCB29DF8083003F00703234325
S1133A4043EAC2239DF80420120202F4E062134305
S1133A509BB2803100EB4111CB805DF8044B704781
S1133A60036813F0800F13D010B400EB411341F23C
S1133A7008041B59002B11DB00EB41131B5913F0F5
S1133A80804F0BD122F0404200EB4110025112E072
S1133A9000EB411041F20803C250704700EB4110A3
S1133AA041F20801435823F47F7323F00303C2F364
S1133AB009021A4342505DF8044B704710B400EBFE
S1133AC0411441F21E03E35A13F4004F14D100EBE6
S1133AD0411141F21E000B5AC2F30E0203F40043DB
S1133AE013430B5241F216000B5A03F400431A43DA
S1133AF00A525DF8044B704741F21E00235AC2F388
S1133B00080203F47E431343235241F21600235A5E
S1133B1003F47E431A432252EBE700EB411241F2D5
S1133B201E03D35A13F4004F07D100EB411041F2A6
S1133B301603C05AC0F30E00704741F21603D05A60
S1133B40C0F30800704700231A46C2540133102BF7
S1133B50FBD1704708B50020FFF710FD08BD08B57C
S1133B600120FFF70BFD08BD08B50220FFF706FD95
S1133B7008BD08B50320FFF701FD08BD08B5042002
S1133B80FFF7FCFC08BD08B50520FFF7F7FC08BDEE
S1133B9008B50620FFF7F2FC08BD08B50720FFF7BB
S1133BA0EDFC08BD08B50820FFF7E8FC08BD08B522
S1133BB00920FFF7E3FC08BD08B50A20FFF7DEFC87
S1133BC008BD08B50B20FFF7D9FC08BD08B50C20CB
S1133BD0FFF7D4FC08BD08B50D20FFF7CFFC08BDE6
S1133BE008B50E20FFF7CAFC08BD08B50F20FFF783
S1133BF0C5FC08BD38B50020FFF7D6FEC56A002411
S1133C0004E06D080134E4B2102C06D015F0010F65
S1133C10F7D02046FFF7C8FCF3E738BD03680B6014
S1133C2043684B6083688B60C3680B6103698B6175
S1133C302C4BDB6CC3F303330F2B4DD8DFE803F0BD
S1133C40080F13171E2125292D3034383C404448D1
S1133C504FF48033CB6000234B61002070474FF05A
S1133C60FF33CB60F7E74FF0FF33CB60F3E74FF45C
S1133C700043CB604FF480534B61EEE70023CB60ED
S1133C80F8E74FF0FF33CB60E5E74FF0FF33CB604D
S1133C90E1E74FF0FF33CB60DDE70023CB60E9E7DA
S1133CA04FF0FF33CB60D6E74FF48043CB60E1E7BE
S1133CB04FF40043CB60DDE74FF48033CB60CAE7B9
S1133CC04FF0FF33CB60C6E74FF0FF33CB60C2E762
S1133CD04FF48033CB60BEE7CB68B3F5803FC9D3E4
S1133CE0B9E700BF008004402DE9F04706461746B7
S1133CF084688C4214D8C3682344994210D201F5D5
S1133D0000010C1B4FF4006808F1FF333B4214BF61
S1133D1001200020194D4FF0700A4FF009091CE0F2
S1133D203468A14224D373682344994223D20C1BE0
S1133D304FF48058E8E785F800A085F80790C4F3AD
S1133D400743AB71C4F307236B71E3B22B713046A5
S1133D5003F0A6FAA7EB080744443FB120B92B7837
S1133D6013F0800FE7D10220BDE8F087BDE8F087AB
S1133D700120BDE8F0870120BDE8F0870000024083
S1133D8038B584688C420DD8C5682544A94209D247
S1133D9001F50001091B144C247814F0800F0AD19A
S1133DA0022038BD0468A1421AD345682544A942BB
S1133DB018D2091BEFE70C4C702525700125E5711D
S1133DC0C1F30745A571C1F307256571C9B2217116
S1133DD0110AE172D2B2A272637203F061FA38BDC1
S1133DE0012038BD012038BD0000024012F0070F49
S1133DF04ED12DE9F04781460C46154682688A4229
S1133E0008D8C16811448C4204D204F50004A41AF1
S1133E1000200CE0D9F80020944207D3D9F804100C
S1133E2011448C4213D2A41A002000E001205E1E2B
S1133E30DFF86C804FF0700A174F5DB350BB98F8F1
S1133E40003013F0800F04D10220BDE8F087012078
S1133E50EDE788F800A0072388F80730C4F3074388
S1133E6088F80630C4F3072388F80530E3B288F8ED
S1133E7004303346094A13F8011F02F8011FBA42FD
S1133E80F9D1484603F00CFA0834083D0836D4E763
S1133E9001207047BDE8F0870F0002400700024090
S1133EA0000002402DE9F04F83B001939DF8349057
S1133EB012F0030F04D00123184603B0BDE8F08FBD
S1133EC0064615468768B94219D3C3683B449942EC
S1133ED015D201F50004E41B4FF0000A5346DFF845
S1133EE0A880DFF8A8B035B12BB998F8003013F0EA
S1133EF0800F0DD102230C9AC2F800A0DCE73768CA
S1133F00B94235D373683B44994235D2CC1BE3E7BD
S1133F10702388F80030022388F80730C4F307437D
S1133F2088F80630C4F3072388F80530E3B288F82C
S1133F30043088F80B90019B5A1E114B12F8011F94
S1133F4003F8011F5B45F9D1304603F0A9F9034694
S1133F5040B10C4A944286BFA7F5000AA24407EB7D
S1133F60040AC0E7043D019A043201920434BAE71A
S1133F704FF0000A0123BEE74FF0000A0123BAE71D
S1133F800B000240FFFF7F00000002400F000240D0
S1133F9010B40B4B0B4C9C420DD02AB100F1100312
S1133FA0084C54F8233013601030064B43F82010AB
S1133FB05DF8044B7047044B044C9C42F8D1ECE789
S1133FC0000000000080FF1F04760000B0720000B3
S1133FD0420900F01F00012303FA00F0014B43F8EB
S1133FE02200704700E100E0430900F01F000122B5
S1133FF002FA00F02033024A42F82300704700BF5F
S113400000E100E0054B1B68002B04DD013B034A83
S11340101360002B00DD704762B6FCE7904E002071
S113402072B6024A1368013313607047904E002041
S1134030002808DB0901C9B200F1604000F56140C5
S113404080F800137047C0B2C0F38102012A0DD07A
S113405010B40A4C0A4B022A18BF234600F003008E
S11340600901C9B219545DF8044B7047054B00F0BF
S113407003000901C9B21954704700BF20ED00E0E4
S11340801CED00E018ED00E030B4C36D44688D7A97
S1134090CA7A954201D030BC70478A69002AFAD0A6
S11340A004F00F0201249440A4B203F007039C42DD
S11340B0F1D94B691B7803664B6901334B618B69FA
S11340C0013B8B61C26D02F00702002BE3D09442E6
S11340D0EFD8E0E7D0F8183123F4706323F0070336
S11340E0C0F81831CB7E3BB98B689BB9D0F81C3132
S11340F023F00103C0F81C31D0F8103123F0010380
S1134100C0F8103100238B700B618B60CB604B6067
S1134110CB757047D0F81C3123F00203C0F81C3172
S1134120EAE7F8B505460C4616461F46836923F4AC
S1134130E05323F00303836191F82730ABB13FB11F
S11341402B6943F480732B612B6943F400732B6157
S113415016B14FF400732B6600236361A361E3601F
S11341602361012384F82230F8BD91F82800FFF779
S11341701BFB236923B1EB6923F00203EB61DEE748
S1134180EB6923F00103EB61D9E738B504460D462A
S1134190C37E3BB1637D4BB1236A13B1616A0420D2
S11341A0984738BD007FFFF7FFFAF3E7214628461A
S11341B0FFF790FFA37E002BEED004F1190002F06C
S11341C039FAE9E730B585B00C460B7C9BB1002287
S11341D02C212078FFF7F4FAA368626861782078CC
S11341E000250395E4680294012401940095FFF7E7
S11341F09DFA05B030BD0022094B13F81010207849
S1134200FFF7DEFA6368A2686178207800250395D9
S1134210E4680294012401940095FFF787FAE8E723
S11342204C72000010B586B0214B53F820406368EF
S113423033B3237F8DF8043001238DF805301D4BF3
S11342400293E368039300238DF8143063680493A6
S113425001A9FFF7B7FF616849429DF80400FFF721
S113426079FB9DF80400FFF793FA6368C3B9124A17
S1134270D2F81C3143F00203C2F81C3106B010BD61
S1134280237F8DF8043000238DF805300B4B029307
S11342902369039301238DF81430A3680493D7E7AB
S11342A0054AD2F81C3143F00103C2F81C31E5E79A
S11342B0984E002060610640006006407061064030
S11342C0474B53F8203093F822300BB90220704743
S11342D0F0B583B017460E46054601A94420FFF702
S11342E031F9404A136923F0010313616FB3019B51
S11342F05A1EF901B2FBF1F20132012A18D9012444
S1134300204600FA04F18A4202D90134072CF8D17C
S113431007FA04F203EB5203B3FBF2F3802B28BF3A
S11343208023012B06D803220227012108461AE024
S11343300024EDE79A1E5108521A49B9032A38BFDE
S113434003220227012108460DE03F2207241146DB
S1134350032A38BF032248080F46022938BF022720
S1134360002808BF01201F4BD3F824C02CF0070CF1
S113437004F0070444EA0C045C629C6C24F07C5452
S1134380000600F07C50204398649C6C24F47C1458
S1134390380400F47C1020439864986C20F47C501A
S11343A0090201F47C5101439964996C21F03F01A5
S11343B002F03F020A439A64094A52F825105A6AE5
S11343C022F0E0625A625A6A22F400725A628E77CC
S11343D01A6942F001021A61002003B0F0BD00BF67
S11343E0944E0020006006402DE9F04107460C463B
S11343F0DFF84C8048F8271000254D618D61CD60B1
S11344000D61012381F82230CD728D720B4E30463E
S113441000F028FAA26BA17F3846FFF751FF218CE8
S113442094F8242058F82730198483F82420336919
S113443043F0010333612846BDE8F0810060064083
S1134440944E002070B505468E4B53F820408E4B99
S11344505B6913F0010F3ED18B4B5B6913F0020FC4
S11344600FD094F83430002B00F0828094F826307A
S1134470002B40F0A8800323A38321462846FFF79E
S1134480B3FF814B5B6913F4805F40F0BB807E4BCC
S11344905B6913F4006F40F0CF807B4B5B6913F4CE
S11344A0806F00F0EE8094F82630002B40F0E0801E
S11344B04FF40073A3830123002221467248FFF7BF
S11344C030FEE36A13B1216B042098474FF48062F5
S11344D06D4B5A6170BDE37AA27A9A4217D163692F
S11344E0002B3FD0A369002B37D194F82320214619
S11344F06548FFF716FE94F826304BBB0023A383D0
S1134500E36A002BA8D0216B04209847A4E75E49F6
S1134510CA6D496801F00F0101268E40B6B202F05F
S11345200702B24298D25849E25C23445B7903EB18
S113453002230B66E37A0133DBB2E372CA6D02F045
S11345400702A07A984200F098809642ECD883E75C
S113455004F1250002F06EF8D0E721464A48FFF73F
S113456093FD79E7484A936923F00103936173E764
S1134570454BDB6D13F4E02F2AD023697BB1424A0B
S1134580E368116F1970E3680133E3602369013B49
S11345902361D16D11F4E02F1AD0002BF0D1002348
S11345A094F8232021463848FFF7BBFD94F82630C1
S11345B01BBB0023A383E36A002B3FF462AF216B90
S11345C0042098475DE704F1250002F033F852E730
S11345D02369002BE3D02C4A926DC2F3014293422B
S11345E03FF64FAF28498A6D22F44032013B1B0449
S11345F003F4403313438B6543E704F1250002F0D1
S113460019F8D6E720484FF4805343610123A3836C
S113461000222146FFF785FD94F826303BB9E36A72
S1134620002B3FF434AF216B042098472FE704F1AB
S1134630250001F0FFFFF2E713484FF400634361E4
S1134640012300222146FFF76CFD94F8263053B96C
S113465040F20323A383E36A002B3FF41EAF216BD4
S11346600420984719E704F1250001F0E3FFEFE780
S113467004F1250001F0DEFF1AE70023E372A372C0
S1134680EAE670BD944E00200060064038B5734BD6
S113469053F82040724BD3F8143113F0040F48D16F
S11346A06F4BD3F8143113F0010F05D06C4BD3F8D2
S11346B0183113F0010F74D1694BD3F8143113F08E
S11346C0020F06D0664BD3F8183113F0020F40F0F6
S11346D08980634BD3F81421D3F8143113F4807F09
S11346E000F0A580E37D0133DBB2E375012B00F01C
S11346F095805B4B4FF40072C3F814214FF4807221
S1134700C3F81421D3F8182122F00102C3F81821A8
S11347102388022B04BF0023238051492046FFF73E
S113472034FD4F4BD3F8143113F4806F40F0848080
S113473038BD05464A4BD3F8503113F0010F1CD055
S1134740236A0BB1627D62B9E37E012B0DD0002395
S11347502376E37EABB9637D9BB12846FFF762FD08
S11347600FE0616A02209847EEE73D4AD2F818311B
S113477043F00103C2F81831E9E7236A3BB1627DD3
S113478012B9022323808BE7616A03209847E37EF2
S1134790002BF6D1637D002BF3D02846FFF742FDB2
S11347A0EFE7237E13B140F20123238063686BB9E2
S11347B0236A23B1616A01209847636833B90123EE
S11347C02376FF22264BC3F8602175E7E3681A7845
S11347D0234BC3F86021E3680133E3606368013B62
S11347E0636069E7A3686BB9236A23B1616A002037
S11347F09847A36833B940F202232380184BD3F8B7
S1134800703166E72369164AD2F870211A70236959
S113481001332361A368013BA3605AE7A37D002B06
S11348203FF467AF4FF480710D4BC3F8141112F4C9
S1134830007F7FF45EAF74E70123238008494FF4BF
S11348408063C1F81431D1F8183123F00103C1F8A1
S113485018312046FFF799FC38BD00BF984E002060
S113486000600640036943F002030361D0F810318D
S113487043F00203C0F8103100230361C0F8103183
S1134880704708B50020FFF7DDFD08BD08B500201E
S1134890FFF7FCFE08BD000070B582B006460C466A
S11348A0264D05EB80014520FEF74CFE002002A9B1
S11348B041F8040DFEF746FE55F82620019B03EB54
S11348C05203B3FBF2F213461D48816841F0020122
S11348D081602AB1013B00BF00BF00BF002BF9D1AA
S11348E017498B6823F002038B601346886840F0F5
S11348F0010088602AB1013B00BF00BF00BF002B4C
S1134900F9D121780E4B9A6822F008029A609A68CD
S1134910002914BF082300231A43094B9A606178C5
S11349209A6822F004029A609B68002914BF04224A
S113493000221343024A936002B070BD9C4E0020D3
S113494000700340024A536919435161704700BF24
S113495000700340F8B506460C461746244D05EB97
S113496080014520FEF7EEFD55F82600214A00237C
S1134970A0FB0701FBF772FD10F1FF3641F1FF3791
S1134980230103F1804303F55C339B6AC3F3810382
S1134990012B20D0022B24D1012F08BF002E12D3CB
S11349A00120F8BD144A0023BB4208BFB24210D311
S11349B0002F08BFB6F5803F05D3B0F101100604FF
S11349C04FF6FF721643023424010C4B1E51002093
S11349D0F8BD0120F8BD012F08BF002EE2D301204D
S11349E0F8BD012F08BF002EEDD30120F8BD00BF94
S11349F09C4E002040420F00FEFF01000070034067
S1134A0030B583B030238DF8043031238DF8053070
S1134A1032238DF8063033238DF807300D4659B90B
S1134A20D37C002B40F0AC80564B996A21F00201F4
S1134A309962996A00230EE0D47C0B0103F1804350
S1134A4003F55C33996A21F002019962996A002C9A
S1134A5014BF02230023144619432B0103F180439E
S1134A6003F55C3399621278996A21F00C0199621A
S1134A70996A920002F00C020A439A626378012B4D
S1134A8068D06168AB1C1B013E4AD150227A2B01CD
S1134A9003F1804303F55C33996A21F400019962C0
S1134AA0996AD20502F400020A439A62E268996A9A
S1134AB021F070619962996A120602F070620A43E9
S1134AC09A62217C9A6A22F480229A629A6A002964
S1134AD014BF4FF4802300231A432B0103F18043B6
S1134AE003F55C339A62617C9A6A22F400329A621A
S1134AF09A6A002914BF4FF4003300231A432B0190
S1134B0003F1804303F55C339A62A17C9A6A22F430
S1134B1080329A629A6A002914BF4FF480330023CA
S1134B201A432B0103F1804303F55C339A62237D1E
S1134B30C3B914490B690122AA4023EA02030B6199
S1134B4002AB1D4415F9040CFFF74EFA0023184676
S1134B5003B030BD62682946FFF7FCFE0346002817
S1134B60F5D193E7074A11690123AB400B43136165
S1134B7002AB1D4415F9040CFFF72AFA0023E6E7FB
S1134B800123E4E700700340014BD960DB68704700
S1134B9000700340036943EA422242EA01220261AF
S1134BA07047B1F57C5F07D04269012303FA01F134
S1134BB01143416100207047436943F47C534361CE
S1134BC0F8E708B5002000F0B5F808BD08B50120E5
S1134BD000F0B0F808BD08B5022000F0ABF808BD3D
S1134BE038B51B4B53F820501A4B53F82040002380
S1134BF02B7395F82430D3B9E36923F00203E361FE
S1134C00E36923F00103E36100F048F9A36923F4A5
S1134C108063A3610A212046FFF7C3FF6B797BB948
S1134C20AB6A1BB1EA6A00212846984738BDA369DC
S1134C3023F00203A361A36923F00103A361E3E763
S1134C4005F1250001F0F6FC00236B71E8E700BFD5
S1134C50A04E0020CC86FF1F10B5084B53F820400F
S1134C60FFF7BEFF012211462046FFF793FF012202
S1134C7011462046FFF78EFF002010BDCC86FF1F93
S1134C8070B50546294B53F82060294B53F8204052
S1134C90636913F4006F0BD033694BB1FFF7DCFF8A
S1134CA00B212046FFF77DFF012386F8263070BDD7
S1134CB0636913F4805F0CD0736953B12846FFF71E
S1134CC0CBFF0C212046FFF76CFF022386F8263029
S1134CD070BD636913F0020F02D0738B9BB2CBB922
S1134CE0636913F0010F02D0338B9BB2B3B9338BDA
S1134CF09BB273B9A36923F00103A361A36943F4CD
S1134D008063A361738B9BB21BB9636913F4806FD7
S1134D1008D170BD284600F07BF8E1E7284600F092
S1134D201DF8E4E72846FFF75BFFF2E7A04E0020FA
S1134D30CC86FF1F02280DD808B5074B53F8203046
S1134D405B6A13F0010F02D100F0FAF808BDFFF717
S1134D5097FF08BD704700BFCC86FF1F2A4B53F84E
S1134D6020302A4A52F82000C26D02F0070293F85C
S1134D702110891A11F0FF0145D0F0B504244FF039
S1134D80000C1FE0026E22F48012026600221A83D5
S1134D90F0BD12F8015B1A61B3F81CE017FA8EFE3D
S1134DA09EFBF6F206FB12E6B6B29E8345661A8BAC
S1134DB0D21B92B21A831A8B92B21AB3013911F030
S1134DC0FF011FD01A791AB11A8B92B2012AD9D0D5
S1134DD05E889A8B92B2B21A042ADDBF9A8BB21AF9
S1134DE097B227461A695AB1012ED2D0022E03D0A7
S1134DF052F8045B1A61CFE732F8025B1A61CBE721
S1134E006546D3E7F0BD7047A04E0020CC86FF1F57
S1134E10F0B4204B53F820101F4B53F82070FE6D54
S1134E20C6F30246002E32D04FF0040C22E0644652
S1134E3000234869DA0025FA02F202704A69013255
S1134E404A6101339AB29442F3D8CB8B14FA83F2B9
S1134E50488892FBF0F300FB13239BB2CB834B8B6C
S1134E601C1BA4B24C834B8B9BB283B1013E16F046
S1134E70FF060CD07D6F4C88CB8B9BB2E31A042BBE
S1134E80D5DCCB8BE41AA4B2002CD1D1DDE7F0BC85
S1134E90704700BFA04E0020CC86FF1F10B50A4B00
S1134EA053F82040A36923F40063A361A36923F4A6
S1134EB08053A3610B212046FFF773FE0C2120468B
S1134EC0FFF76FFE10BD00BFCC86FF1F38B51A4B2D
S1134ED053F82040194B53F8205095F82430012BF7
S1134EE019D0E36923F00203E361E36923F00103CA
S1134EF0E361FFF7D3FF00232B7301221146204601
S1134F00FFF748FE012211462046FFF743FE6B7966
S1134F1053B9002038BDA36923F00103A361A36939
S1134F2023F00203A361E4E705F1250001F082FB0D
S1134F3000236B71EDE700BFCC86FF1FA04E00205D
S1134F4070B50646314B53F82050314B53F820408E
S1134F506B6913F4006F07D023692BB1FFF7B6FF19
S1134F60012384F8263070BD6B6913F4805F08D088
S1134F70636933B13046FFF7A9FF022384F8263072
S1134F8070BD6B6913F0020F03D0638B9BB2002BCF
S1134F902DD16B6913F0010F02D0238B9BB253BB4D
S1134FA0238B9BB21BB9AB6923F00103AB61638B09
S1134FB09BB21BB9AB6923F00203AB61638B9BB259
S1134FC0A3B9238B9BB28BB9AB6923F40063AB61A8
S1134FD0AB6923F48053AB61A36A1BB1E26A00217D
S1134FE020469847637953B90023237370BD304634
S1134FF0FFF70EFFCDE73046FFF7B0FED0E704F130
S1135000250001F017FB00236371EDE7CC86FF1F39
S1135010A04E002038B5144B53F82040134B53F8DE
S11350202050EB8D9BB2022B16D000221049204653
S113503000F029FD00220F49204600F024FDA36959
S113504023F40023A361A36913F4002FFBD10023ED
S11350502B74AB7C1BB938BD0023EB85EAE705F163
S11350602C0001F0E7FAF6E750720000AC4E002085
S1135070170003001600030038B5154B53F8204001
S1135080144B53F82050236923F40003236195F84B
S11350902A00FEF789FB00220F49204600F0F3FCAA
S11350A0A36923F40023A361A36913F4002FFBD1A4
S11350B0AB7C43B9EB8D9BB2022B04BF0023EB8581
S11350C000232B7438BD05F12C0001F0B3FAF1E78D
S11350D050720000AC4E00201600030008B50E4BC1
S11350E053F820300D4A52F820001A681B7D43B152
S11350F0012B09D01378517843EA012100F09AFC7E
S113510008BD1378037708BD1378517843EA012169
S113511000F085FC08BD00BFAC4E002050720000BA
S113512010B5114B53F820305C7C0CB1022010BD3B
S11351300E4C54F82040012058745960DA60022261
S11351401A86A36943F48023A361A36913F4802F0F
S1135150FBD00121204600F0AFFD01220449204686
S113516000F091FC002010BDAC4E002050720000F5
S1135170150003002DE9F04385B0244C54F8205069
S11351806C7C1CB1022005B0BDE8F0830F460646D6
S11351901F4B53F8204095F829004FF00108CDF833
S11351A00C800292CDF804804FF00009CDF80090F5
S11351B00B4604F11C024946FEF7B8FA324615497B
S11351C095F82900FEF7CAF995F82900FEF7E0FAE8
S11351D06F60C5F80C9085F8118002232B86A369B3
S11351E043F48023A361A36913F4802FFBD001212E
S11351F0204600F061FD01220749204600F043FCEF
S1135200236943F4001323610020BCE7AC4E002063
S113521050720000E55200001400030038B5154B2D
S113522053F82050144B53F82040A36923F48023EF
S1135230A361A36913F4802FFBD10021204600F061
S11352403BFDE36900220D49204600F01CFCEB7C89
S113525043B900236B742B8E9BB2022B04BF002333
S11352602B8638BD05F12B0001F0E4F90023EB7423
S1135270EFE700BFAC4E00205072000015000300A1
S113528038B5164B53F82040154B53F82050A369FA
S113529023F48023A361A36913F4802FFBD100219D
S11352A0204600F009FD236923F400132361E36918
S11352B095F82900FEF778FAEB7C43B92B8E9BB264
S11352C0022B04BF00232B8600236B7438BD05F129
S11352D02B0001F0AFF90023EB74EFE750720000EC
S11352E0AC4E002070B50546254B53F82040254BA5
S11352F053F82060012904D0238E9BB2022B13D0D3
S113530070BD01232386FFF7BBFFA3691BB1E269CC
S1135310032120469847736923F0C02323F4F8132C
S113532043F470237361E7E7A3691BB1E2690021C9
S113533020469847E3688BB92846FFF7A1FFA36985
S11353401BB1E269022120469847736923F0C02308
S113535023F4F81343F470237361D1E7616894F87C
S11353602900FEF702FBE16894F82900FEF708FB28
S11353700023E36094F82900FEF70AFA70BD00BF29
S1135380AC4E00205072000010B582B0134B53F89D
S11353902030134A52F820005C681B7D73B1012B46
S11353A00FD00DF1060100F05FFBBDF8063023704D
S11353B0BDF806301B0A637002B010BDC3692370C8
S11353C0FAE70DF1060100F046FBBDF80630237044
S11353D0BDF806301B0A6370EEE700BFAC4E002038
S11353E050720000034B53F8203098699961DA61D8
S11353F0704700BFAC4E0020034B53F82030186AAE
S113540019625A62704700BFAC4E00202DE9F84380
S11354101C4B53F8208098F8103013B10220BDE8DB
S1135420F88381460F461646174B53F82040A3696C
S113543043F40023A361A36913F4002FFBD0B6B196
S1135440124D02E00237023E8EB12946204600F09A
S113545077FB0028F9D0C8F800704846FFF73EFEF5
S113546098F81430002BEDD10137013EECE7A36925
S113547023F40023A361A36913F4002FFBD10020BC
S1135480BDE8F883AC4E0020507200001700020003
S113549010B5074B53F820300024DC7493F82830FF
S11354A0012B02D0FFF766FE10BDFFF739FE10BDD9
S11354B0AC4E0020384B53F820303BB11A7C0AB173
S11354C0022070475B7C0BB1022070472DE9F0414C
S11354D082B00C46314B53F8205001A9304B185C74
S11354E0FEF730F801984FEA840CB0FBFCFC1FFA7D
S11354F08CFC4FEA8C07B0FBF7F7BC4234BF3F1B70
S1135500E71BB0FBF4F8B8F1200F28BF4FF02008D8
S1135510B8F1040F38D905264FF0040E324604E0E2
S1135520013292B21646424513D806FB04F1B0FB91
S1135530F1F18BB202FB03F3B0FBF3F39C4234BFF3
S11355401B1BE31ABB42EBD81FFA81FC1F46B6466D
S1135550E6E7BEF1070F19D92A6922F0F8520EF1D5
S1135560FF331B0603F0F85313432B612B6923F419
S1135570FF5323F01F03CCF30C0C4CEA03032B6101
S1135580002002B0BDE8F0814FF0040E2B6943F413
S113559000332B61E0E700BFAC4E002050720000E6
S11355A05C720000F0B583B007460C461646354BD6
S11355B053F8205001A9344B185CFDF7C3FF631E58
S11355C004F13301002203F8012F8B42FBD12F4B4E
S11355D043F82740F37984F82830B3792375337A74
S11355E084F82930737A84F82A30284600F0DEF9EA
S11355F031683846FFF75EFF3379002B3AD0012239
S1135600B179284600F0E4F93179284600F0F8F938
S11356102B69727923F4005343EA42332B61AB695B
S113562023F4E06343F44073AB61AB6943F00403D8
S1135630AB610025E5852586294604F12B0001F0A0
S11356400CF80646294604F12C0001F006F8012E58
S113565016D001280CD00E4BDC572A460D4B53F8BC
S113566027102046FEF794FC2046FEF7B1FC28469E
S113567003B0F0BD0022B179284600F0A9F9C3E7D0
S11356803046F5E7507200005C720000AC4E00201A
S113569060720000D886FF1F034B53F82030596016
S11356A0DA600020704700BFAC4E0020F8B5064613
S11356B09D4B53F820409D49204600F01CFA0028D9
S11356C036D19B4B53F826509A49204600F038FABD
S11356D0002850D040F201632B8695F82830012B26
S11356E045D03046FFF7CCFDAB691BB1EA69032115
S11356F028469847636923F0C02323F4F81343F43E
S1135700702363618C49204600F0F5F9002840F0CD
S11357109B808A49204600F0EEF9002840F0C880BA
S11357208749204600F0E7F9002840F01981F8BDC8
S11357308449204600F004FA0028C2D07C4B53F878
S113574026508049204600F01FFA95F82830002B97
S1135750B7D195F82900FEF71DF9E8603046FFF748
S11357608FFDAB690022042128469847A9E73046FB
S1135770FFF754FDB8E77449204600F0E1F9E0B1C1
S113578040F203632B8695F82830012B11D0304664
S1135790FFF776FDAB691BB1EA69032128469847F8
S11357A0636923F0C02323F4F81343F47023636183
S11357B0A8E73046FFF732FDECE76449204600F0E5
S11357C0BFF9E0B140F204632B8695F82830012B31
S11357D011D03046FFF754FDAB691BB1EA690321D0
S11357E028469847636923F0C02323F4F81343F44D
S11357F07023636186E73046FFF710FDECE75449F8
S1135800204600F09DF9E0B140F205632B8695F83F
S11358102830012B11D03046FFF732FDAB691BB1A4
S1135820EA69032128469847636923F0C02323F4D7
S1135830F81343F47023636164E73046FFF7EEFC2A
S1135840ECE7444B63615DE74349204600F078F997
S113585000283FF45EAF364B53F826503046FFF72E
S113586093FD2B7DEBB96B6801336B60EB68013BF7
S1135870EB60EB682BB9AB691BB1EA6900212846E0
S11358809847EB68002B7FF444AF3046FFF7C6FC23
S1135890AB69002B3FF43DAFEA69022128469847E3
S11358A037E76B6802336B60EB68023BEB60E0E761
S11358B02A49204600F044F900283FF431AF1C4B3C
S11358C053F82650AB68002B3FF42AAF164B53F81D
S11358D026703046FFF702FC2B7DF3B92B680133A9
S11358E02B60AB68013BAB60AB68002B7FF418AF57
S11358F02B6A1BB16A6A012128469847AB68002BC2
S11359007FF40EAF00220D49384600F0BCF80122A6
S11359100B49384600F0B7F802E72B6802332B60D6
S1135920AB68023BAB60DFE7507200001400030079
S1135930AC4E002013000200150003001700030002
S113594016000300140002001100020010000200FF
S11359501200020000C01FC0150002001700020060
S11359601049204600F0ECF800283FF4E0AE0E4B5E
S113597053F82640A368002B7FF4D9AE94F828305E
S1135980012B0BD03046FFF777FB236A002B3FF443
S1135990CEAE626A022120469847C8E63046FFF739
S11359A039FBF2E716000200AC4E0020064B0361FF
S11359B0064B436100238361036243624FF47032F8
S11359C08262C362704700BF0400000F00C01FC0A2
S11359D010B40C4602B14C1C022C0CD0836923F089
S11359E0100343EA04138361036923F00053036142
S11359F05DF8044B7047036943F000530361F7E714
S1135A00826901F0FE0322F0020213438361836979
S1135A1023F0010301F00101194381617047836997
S1135A20C1F3002223F0804343EA82738361C9B245
S1135A3001777047836923F08043C1F3002243EA6E
S1135A40827323F00043C1F3402243EAC2738361AB
S1135A50C9B2017770478369DB0F1B020B80C269EF
S1135A60D2B213430B80704783695B0D03F4007358
S1135A700B808269D20F43EA02230B80C269D2B23F
S1135A8013430B80704710B48BB2090C01390629FB
S1135A900ED8DFE801F0040D100D0D1A2400016981
S1135AA001249C4021EA040102FA03F30B4303613D
S1135AB05DF8044B7047816901249C4021EA04018C
S1135AC002FA03F30B438361F2E7416A01249C4029
S1135AD021EA040102FA03F30B434362E8E7816A13
S1135AE001249C4021F4403121EA040102FA03F329
S1135AF00B438362DCE70B0C013B062B1ED8DFE86B
S1135B0003F0041D0B1D1D111700036988B223FA4D
S1135B1000F000F001007047806989B2C84000F0CD
S1135B2001007047406A89B2C84000F00100704724
S1135B30806A89B2C84000F00100704700207047B5
S1135B400B0C023B052B1DD8DFE803F0031C0A1CD9
S1135B501016436988B223FA00F000F00100704780
S1135B60C06989B2C84000F001007047406A89B238
S1135B70C84000F001007047806A89B2C84000F054
S1135B800100704700207047474B994250D023D8FA
S1135B90033B994260D00FD8023B994270D0013345
S1135BA099427FD1436923F0C02323F4F81343F4CB
S1135BB000434361002070473C4B994242D001337B
S1135BC099426FD1436923F0C02323F4F81343F4BB
S1135BD08023436100207047354B994246D00FD84B
S1135BE00B3B99421AD00A3399425BD1436923F0A3
S1135BF0C02323F4F81343F080434361002070472B
S1135C002C4B994246D0013399424BD1836A23F4F9
S1135C10403343F40033836200207047436923F028
S1135C20C02323F4F81343F4801343610020704726
S1135C30436923F0C02323F4F81343F4002343619E
S1135C4000207047436923F0C02323F4F81343F47E
S1135C500033436100207047436923F0C02323F4D9
S1135C60F81343F48033436100207047436923F001
S1135C70C02323F4F81343F000434361002070472A
S1135C80436923F0C02323F4F81343F480434361AE
S1135C9000207047836A23F4403343F480338362E3
S1135CA00020704701207047130002001100020019
S1135CB01F0002001000070038B505460C460A46CE
S1135CC00949FFF7E0FE224608492846FFF7DBFEB4
S1135CD0224607492846FFF7D6FE224605492846AC
S1135CE0FFF7D1FE38BD00BF1B00030018000300FE
S1135CF01A0003001900030008B50020FFF7D6FCC2
S1135D0008BD08B50120FFF7D1FC08BD08B5022085
S1135D10FFF7CCFC08BD60B170B506460C46002503
S1135D20204600F041F801351834AE42F8D1002085
S1135D3070BD002070470000194B984204D0194BE5
S1135D40984220D0FF207047102927D8DFE801F0BF
S1135D50090C26262626262626262626260F121552
S1135D60180042F00100704742F00200704742F010
S1135D700400704742F00800704702F00E007047BC
S1135D8002F00D00704719B1012904D0FF207047BB
S1135D9002F00B00704702F007007047FF207047C5
S1135DA000A0044000B0044038B5044600686168AF
S1135DB050F82120237A012B3FD0002B3AD0022B1C
S1135DC040D0657A2D0105F0100322F050051D43E3
S1135DD0A37A9B0103F040032B4323F4E065E37AA9
S1135DE0082B32D01B0203F4E0632B43227BD20343
S1135DF092B223F478231343627B120402F47022D8
S1135E001343A27B0AB143F080732268616842F8AD
S1135E1021302168D1F8C02060680123834022EA40
S1135E200302E37B83401343C1F8C030E37A012BC0
S1135E3021D038BD22F00202C3E722F0010242F071
S1135E400202BEE742F00302BBE71B4B5A6802F0B2
S1135E500F02FFF771FFFF280BD0174B5A6822F08F
S1135E600F025A605A6800F00F0010435860002374
S1135E70B8E70023B6E721694B69227D22B1012AE4
S1135E800AD0012A05D10BE0616801228A4023EA85
S1135E90020322695361CCE7606801228240134304
S1135EA0656808680122AA4020EA0200627DAA40CF
S1135EB002430A60EDE700BF00800440124BD3F8B0
S1135EC0003623F00103114A12780AB143F00103AA
S1135ED00D4AC2F80036D2F8003323F001030C4A0D
S1135EE012780AB143F00103074AC2F80033D2F82A
S1135EF0003123F00103074A12780AB143F0010389
S1135F00014AC2F80031704700400640BB4E0020F1
S1135F10B94E0020BA4E0020094BD3F8002622F0D7
S1135F200102C3F80026D3F8002122F00102C3F8CD
S1135F300021D3F8002322F00102C3F800237047A4
S1135F40004006400378042B13D000B583B004232B
S1135F508DF800300123ADF802300223ADF804308F
S1135F60ADF8063069460020FDF7BAF903B05DF8D4
S1135F7004FB00207047000010B582B000238DF8A8
S1135F8005308DF804301E4B1A79CAB11868031F06
S1135F90013AD2B200EB8200012406E01278022A10
S1135FA00BD0052A09D083420AD053F8042F117864
S1135FB00029F3D18DF80540F0E78DF80440F2E7AD
S1135FC0104A937803F0FE03937001A90E4800F081
S1135FD075FA0E4BD3F8002602F001020C490A7040
S1135FE0D3F8002302F001020A490A70D3F8003101
S1135FF003F00103084A1370002002B010BD00BF73
S1136000BC4E002000D0074000E00740004006409E
S1136010BB4E0020B94E0020BA4E0020074B5B69EE
S1136020DBB2042B06D0802B06D0012B0CBF012041
S113603006207047022070470020704700E00740A8
S113604030B583B00378022B16D90546B04A52699D
S1136050D2B2042A00F0C680102A00F00C81012A72
S113606000F06781032B05D3042B40F20D81052B2F
S113607000F0C88004242DE1A54A5269D2B2042A52
S113608000F0EF800DD8012A00F02B81022A40F0A5
S11360905C810222012B55D093B1022B6FD00424D2
S11360A018E1102A00F04F81802A40F04E81012B24
S11360B03CD00BB900240DE1022B5DD0042409E18E
S11360C002A9012301F8083D914800F079F904463A
S11360D0002840F0FF8008E10124FBE0062B02D0F9
S11360E08C4B1B7803B38C4B1B78A3B1FFF7E6FEF4
S11360F08A490020FDF7F4F80446002840F0EA80BD
S11361000023854A137002A901F8043D804800F079
S113611057F90446DEE002A9002301F8043D7C4857
S113612000F04EF90446D5E00124D3E0802300E0DA
S11361300423012B06D1784B1B787BB90024C9E0DA
S11361400123F6E702A9012301F8083D704800F095
S113615037F90446002840F0BD80ECE7FFF7AEFEB7
S11361606E490020FDF7BCF80446002840F0B280D8
S11361700022694B1A70ADE0802200E00422042A58
S11361802ED0634B5B69DBB2012B0AD002A9012339
S113619001F8083D5E4800F013F90446002840F079
S11361A099805D4B1B78BBB15C48FFF7CBFE04467E
S11361B0002840F08F800122574B1A7002AC022352
S11361C004F8083DFFF7A8FE2146514800F0F8F80E
S11361D004467FE00122D2E75048FDF703F9E3E7E4
S11361E0002477E0032B3AD3042B07D9052B36D1AF
S11361F0FFF714FF012813D000240DE004233FE02F
S113620001233DE002A9012301F8043D404800F0C8
S1136210D7F804460028EBD005238DF8043044E079
S11362203D4B1B7873B13D48FFF78CFE04460028B4
S1136230F2D10122384B1A7005238DF80430FFF790
S11362406BFEE9E73548FDF7CDF8ECE74FF0E022C7
S1136250D2F8103D23F00203C2F8103D31E00424CB
S113626038E0012B3FF464AF002B3FF429AF022B3D
S113627084D004242EE0032B31D3042B2DD81023F7
S1136280012B08BF002407D002A9012301F8043D13
S11362901F4800F095F804462B788DF80430032B42
S11362A00CBF012302238DF805309CB96B78002BB9
S11362B0CCD04FF0E022D2F8103D43F00203C2F8F4
S11362C0103D01A9124800F07BF8041E40F20113AE
S11362D018BF1C46204603B030BD052B92D00424C1
S11362E0F8E7012B3FF42CAFF3B90D4BDB69C3F393
S11362F003630C4A1278002A7FF4F0AE054A127840
S1136300002A3FF4E9AE062B7FF4EAAE0124E1E76C
S113631000E00740B94E0020B84E0020CC4E0020CB
S113632000400640BB4E0020022B3FF453AF042430
S1136330D0E7032B05D3042B7FF662AF052B3FF484
S113634057AF0424C6E71022A4E6FF22A2E600BF4A
S11363502DE9F04180290BD05AB300244FF00408F2
S11363604FF0FF0E4FF0100C8027012602250FE09E
S11363706423013BFDD1EFE7102B16D0802B10D105
S11363803B4600E02B46994214D00134A24211D07E
S11363904369DBB2042B06D0EED8012B07D0022BC5
S11363A0F0D07346EFE74346EDE76346EBE7334649
S11363B0E9E70024A24294BF00200120BDE8F08157
S11363C008B50B78052B75D8DFE803F02F031743C6
S11363D04343394A937803F0FE039370C36823F070
S11363E06003C3604FF47A720121FFF7B1FF002804
S11363F040F2011018BF002008BD2F4A937803F023
S1136400FE0343F001039370C36823F0600343F079
S11364104003C3604FF47A720421FFF799FF002808
S113642040F2011018BF002008BD234A937803F0FE
S1136430FE039370C36843F06003C3604FF47A7241
S11364408021FFF785FF002840F2011018BF0020CB
S113645008BD033BDBB2012B22D9174A937803F022
S1136460FE0343F0010393700223C26822F0070283
S11364701343C3604FF0E022D2F8103D43F004030D
S1136480C2F8103D30BF4369DBB2012B0A4A93784E
S113649003F0FE0318BF43F001039370002008BD0E
S11364A0026922F0C0024B789B01DBB21343036103
S11364B00023DAE7042008BD00D007400B78002B46
S11364C00CBF002320234A780AB143F08003836081
S11364D0704700002DE9F04F83B08379012B07D07A
S11364E0EBB1022B15D001274FF0000B5E4604E000
S11364F0204B1E7B022740F2031B00230B70002E4F
S11365002FD091460C4680469A461A4DCDF804B0D9
S113651011E0184B1E7B01274FF4827BEDE7154BEE
S11365201E7B022740F2031BE7E723780133DBB22B
S113653023709E4219D9AA6852F82330002BF4D054
S11365401A79BA42F1D01A689968404690470028EF
S1136550EBD023786B73B9F1010F05D1DDF804A0FA
S1136560E3E74FF0000A00E0DA46504603B0BDE826
S1136570F08F00BFBC4E002010B5094C2060217183
S11365800021A17332B11146A16023736373FFF735
S1136590F3FC10BD024B00229A601A735A73F6E79B
S11365A0BC4E0020F0B585B006460C4600238DF89D
S11365B00F301B4B1A6852F820701A7B5A738DF8EF
S11365C009108DF80800019701238DF80A300A4656
S11365D00DF10F0101A8FFF77DFF012C01D0054645
S11365E088B93846FFF72CFD054660B90C4B9E73FD
S11365F002238DF80A3001220DF10F0101A8FFF7E3
S113660069FF054608E000238DF80A3001220DF1E8
S11366100F0101A8FFF75EFF284605B0F0BD00BFDB
S1136620BC4E0020024A136801331360704700BF58
S1136630D44E002010B50446FDF7F2FC2378DBB2FB
S1136640FF2B08D023780133DBB223700024FDF73D
S1136650D9FC204610BD0124F9E738B504460D469F
S1136660FDF7DEFC2570FDF7CDFC002038BD0000F1
S113667008B5FAF779FFFAF73BFE054A1368002BD1
S1136680FCD0034A1368002BFCD0014B186808BDEA
S1136690DC4E002010B5431E0A44914200D110BDC7
S11366A011F8014B03F8014FF7E702440346934204
S11366B000D1704703F8011BF9E710B59AB04FF405
S11366C00274019105916FF00041039106914FF618
S11366D0FF71ADF8121001A9ADF8104000F06CF88C
S11366E0019B00221A701AB010BD000013460A461E
S11366F0014602480068FFF7E0BF00BFF086FF1FB5
S11367002DE9F0478E689E4282460C469146984693
S113671035D88A8912F4906F31D0256809696F1AC7
S11367206569022305EB450595FBF3F508F10103C3
S11367303B449D4238BF1D46530531D5294600F0E0
S11367402DFB064650B90C23CAF80030A38943F048
S11367504003A3814FF0FF30BDE8F0873A4621693A
S1136760FFF798FFA38923F4906343F08003A38188
S1136770266165613E44ED1B2660A560464646459C
S113678028BF464632464946206800F09FFAA3686F
S11367909B1BA36023681E4426600020BDE8F0878D
S11367A02A4600F059FB06460028E1D121695046EB
S11367B000F0A6FAC7E700002DE9F04F9DB080462F
S11367C003938B891C060D4616460FD50B696BB9CE
S11367D0402100F0E3FA2860286128B90C23C8F8A6
S11367E000304FF0FF30C5E040236B610023099374
S11367F020238DF8293030238DF82A304FF0010BF7
S113680037463C4614F8013B002B3CD1B7EB060A53
S11368100BD05346324629464046FFF771FF0130FC
S113682000F0A380099B534409933B78002B00F0AC
S11368309C8000234FF0FF32049307930592069344
S11368408DF853301A93052221785048F9F798FFB0
S1136850671C049BD8B9D90644BF20228DF8532065
S11368601A0744BF2B228DF8532022782A2A16D0E7
S1136870079A00210A20274601343B78303B092B34
S113688051D9C9B111E0252BC0D02746B9E73F4AF9
S1136890801A0BFA00F0184304903C46D3E7039A9D
S11368A0111D12680391002A01DB079204E0524291
S11368B043F00203079204933B782E2B0ED17B788E
S11368C02A2B07F1010132D1039B1A1D1B68039285
S11368D0002BB8BF4FF0FF33023705932C4C3978A7
S11368E003222046F9F74CFF38B14023001B03FA7A
S11368F000F0049B034304930137397825488DF84D
S1136900281006227E1CF9F73BFF002835D0224BC5
S1136910FBB9039B073323F0070308330393099B55
S11369204B4409936CE700FB02320121A3E70023E7
S1136930059318460A240F4601313A78303A092A59
S113694003D9002BCAD00590C8E704FB002001231B
S1136950F1E703AB00932A46104B04A94046AFF37A
S11369600080B0F1FF3F8146D9D1AB895B063FF58A
S113697038AF09981DB0BDE8F08F03AB00932A46E9
S1136980064B04A9404600F081F8EAE76372000070
S1136990697200006D7200000000000001670000D1
S11369A02DE9F04791461F468A680B69DDF820807F
S11369B09342B8BF1346C9F8003091F84320064605
S11369C00C4612B10133C9F800302368990642BF5E
S11369D0D9F800300233C9F80030256815F00605EF
S11369E007D104F1190AE368D9F800209B1A9D42E3
S11369F029DB94F843302268003318BF0123920640
S1136A002ED404F1430239463046C047013021D028
S1136A102368E568D9F8002003F00603042B08BFB7
S1136A20AD1AA36822690CBF25EAE57500259342D7
S1136A30C4BF9B1AED184FF000091A344D451BD101
S1136A400020BDE8F0870123524639463046C0474E
S1136A50013003D14FF0FF30BDE8F0870135C2E7C4
S1136A60E1185A1C302081F84300224494F8451060
S1136A7082F843100233C4E70123224639463046E4
S1136A80C0470130E6D009F10109D7E72DE9F04309
S1136A9017460A7E85B06E2A984606460C460C9B1D
S1136AA001F1430C00F0BC801AD8632A2ED00AD816
S1136AB0002A00F0C880582A00F08A8004F14205B8
S1136AC084F842202AE0642A01D0692AF6D1216898
S1136AD01A6811F0800F23D0111D1960136827E084
S1136AE0732A00F0B48008D86F2A2AD0702AE5D11E
S1136AF00A6842F020020A6003E0752A21D0782A4D
S1136B00DCD1782284F845206E4964E01A6801F1EA
S1136B104205111D1960136884F842300123A3E073
S1136B2011F0400F02F104011960D7D0B2F900301E
S1136B30002B03DA2D225B4284F8432062490A22A7
S1136B4017E02068196810F0800F03D0081D186042
S1136B500B6806E010F0400F01F104001860F7D054
S1136B600B8859496F2A14BF0A220822002084F88E
S1136B7043006568A560002DC0F29C80206820F069
S1136B8004002060002B3FD1002D40F09580654625
S1136B90082A0BD12368DA0708D5236962689A4268
S1136BA0DEBF302305F8013C05F1FF35ACEB0503EE
S1136BB02361CDF800803B4603AA21463046FFF707
S1136BC0EFFE013055D14FF0FF3005B0BDE8F08342
S1136BD081F845203C492268186812F0800F00F1C2
S1136BE004051D6001D0036802E05506FBD5038847
S1136BF0D00744BF42F0200222601BB9226822F071
S1136C00200222601022B1E76546B3FBF2F002FBDA
S1136C101033CB5C05F8013D03460028F5D1B7E7F6
S1136C2008681A68496910F0800F04D0101D1860B4
S1136C301368196007E010F0400F02F104001860B7
S1136C401368F6D01980002323616546B1E71A68FA
S1136C50111D19601568626800212846F9F790FD36
S1136C6008B1401B606063682361002384F84330EB
S1136C709FE723692A4639463046C0470130A2D0EF
S1136C8023689B0707D5002504F11909E368039AD3
S1136C909B1A9D4205DBE068039B9842B8BF1846E7
S1136CA093E701234A4639463046C04701308AD02B
S1136CB00135EBE7002BA7D10B7884F8423004F1BF
S1136CC0420565E78572000074720000884210B5C1
S1136CD001EB020303D8421E99420CD110BD984225
S1136CE0F9D28118D21AD34200D110BD13F8014D44
S1136CF001F8014DF7E711F8014B02F8014FEBE7FA
S1136D0038B50546002945D051F8043C0C1F002B2A
S1136D10B8BFE41800F0D6F81F4A1368104633B918
S1136D20636014602846BDE8384000F0CCB8A34244
S1136D300CD921686218934204BF1A685B686360C7
S1136D4004BF521822600460ECE713465A680AB183
S1136D50A242FAD919685818A0420BD120680144FC
S1136D60581882421960DDD1106852685A60014493
S1136D701960D7E702D90C232B60D3E720682118C8
S1136D808A4204BF11685268626004BF0918216016
S1136D905C60C7E738BD00BFF85E002070B5CD1C4D
S1136DA025F0030508350C2D38BF0C25002D0646AB
S1136DB001DBA94203D90C233360002070BD00F02D
S1136DC081F8234A1468214691B9224C23681BB9DF
S1136DD0304600F067F820602946304600F062F83B
S1136DE0431C26D10C233360304600F06CF8E4E7F2
S1136DF00B685B1B1AD40B2B0FD90B60CD50CC182E
S1136E00304600F060F804F10B00231D20F0070069
S1136E10C31A1BD05A42E25070BD8C420DBF636846
S1136E204B686360136018BF0C46E9E70C46496879
S1136E30CAE7C41C24F00304A04205D0211A30463A
S1136E4000F030F80130CDD02560D9E770BD00BF27
S1136E50F85E0020FC5E0020F8B5074614460E4696
S1136E6021B91146BDE8F840FFF798BF22B9FFF7F2
S1136E7047FF25462846F8BD00F026F884420FD97E
S1136E8021463846FFF78AFF05460028F2D03146EE
S1136E902246FFF7FFFB31463846FFF731FFE9E7AB
S1136EA03546E7E738B5064C002305460846236017
S1136EB000F014F8431C02D1236803B12B6038BDE1
S1136EC0045F00207047704751F8040C0028A0F1BB
S1136ED00400BCBF0B58C01870470000044B19686D
S1136EE0024609B903491960186802441A607047D8
S1136EF0005F0020085F0020200D0A0D0A2D2D2DB3
S1136F002D5333324B31343420626F6F746C6F61A4
S1136F106465722056657273696F6E203230323048
S1136F202F30372F3039202D2D2D2D2D2D2D2D2D7A
S1136F302D310D0A00000000200D0A0D0A2D2D2D03
S1136F402D5333324B31343420626F6F746C6F6164
S1136F506465722056657273696F6E203230323008
S1136F602F30372F3039202D2D2D2D2D2D2D2D2D3A
S1136F702D32200D0A0000000D0A205333324B201D
S1136F80626F6F745F75617274206261756472619F
S1136F907465206973203A202564206269742F7314
S1136FA0200D0A00AC2C0020CC3C0020EC4C00202E
S1136FB00484FF1F0584FF1F0684FF1F00000000D8
S1136FC0000008000000001000000014FFFFFFFF95
S1136FD000000000CC84FF1FDC84FF1FEC84FF1F33
S1136FE0FC84FF1F0C85FF1F1C85FF1F2C85FF1FC2
S1136FF03C85FF1F084D0020184D0020284D00201F
S1137000384D0020484D0020584D0020684D002088
S1137010784D002000000000C0C62D0000000001D3
S11370200000000000C20100000000000405000090
S113703000100E000000000100000000000000002D
S1137040000000000000000000000000000000003C
S1137050000000000000000000000000000000002C
S1137060000000000000000000000000000000001C
S1137070000000000000000000000000000000000C
S11370800000000000000000000000000000730089
S113709032002100610049004A004B004C004D00C1
S11370A03D000000240025002B00360031000000C4
S11370B020000000380039003A00260000003B00A0
S11370C027005A00660037002C002D002E004000D7
S11370D06A006B006C00000000000000000000006B
S11370E0000000000000000000FCAC06007E560317
S11370F0003FAB0100FCAC06007E5603003FAB0131
S113710000FCAC06007E5603003FAB01000000000B
S1137110000000000000000000000000000000006B
S11371200000000000FCAC06007E5603003FAB01EB
S113713000000000000000000000000000B4C404CF
S1137140006CDC02B0F3960100B4C404006CDC02F1
S1137150B0F3960100B4C404006CDC02B0F39601F1
S1137160000000000000000000000000000000001B
S1137170000000000000000000B4C404005A6202D1
S1137180B0F39601000000000000000000000000C1
S113719000093D0000093D0040420F0000093D0088
S11371A000093D0040420F0000093D0000093D0078
S11371B040420F000000000000000000000000003A
S11371C000000000000000000000000000093D0075
S11371D000093D0040420F000000000000000000D4
S11371E0000000000000000000000000000000009B
S11371F00000000000000041414141410000000046
S1137200002020202020202020202000404040403A
S1137210400080004848484800303030303030303A
S1137220303630303000000000000102030405064F
S11372300708090A0B0C0D0E0F00000000010203E1
S11372400405060708090A0B0C0D0E0F2D2C00006F
S113725000A0064000B0064000C006404A4B4C0067
S11372601F2123232D302B2000686C4C006566679A
S113727045464700303132333435363738394142A8
S1137280434445460030313233343536373839617A
S11372906263646566000000F8B500BFF8B500BF1E
S10B72A05FF800F00988FF1FEC
S10B72A8E491FF7F01000000E6
S11372B001000000010101000101010101010000C0
S11372C0010100000100010000127A000001000326
S11372D0010100000001000000000C000101000099
S11372E00100000000000000010000000301010192
S11372F00003030001020301000600010100000075
S11373000100000101000000010000000000000075
S11373100000000000000000010101010101010161
S1137320000000000E0000008484FF1F0101000023
S11373300884FF1F2B0100000044010600004501E2
S11373400600004601030000470103000048010352
S113735000004A010600004B010600004C01060033
S1137360002D010000002E010000002F010000008C
S1137370300100000031010000000000FF000E0099
S1137380000000000000000000000000FF010F00EA
S1137390000000000000000000000000FF020200E6
S11373A0000000000000000000000000FF030300D4
S11373B0000000000000000000000000FF040400C2
S11373C0000000000000000000000000FF050500B0
S11373D0000000000000000000000000FF0606009E
S11373E0000000000000000000000000FF0707008C
S11373F00000000000000000000000000001000088
S11374006400000001000000000000000000000013
S11374100100000000010000F40100000100000070
S11374200000000000000000010000000001000056
S11374301027000001000000000000000000000010
S11374400100000000010000A0860100010000000E
S113745000000000000000000100000000C0044023
S1137460100000000000000100000000C0F00F4008
S1137470010100000090044003000000000000032C
S11374800000000000000000000000000090044024
S113749002000000000000030000000000000000E3
S11374A00000000000B004400700000000000002DB
S11374B000000000000000000000000000B00440D4
S11374C006000000000000020000000000000000B0
S11374D0000000002886FF1F010000004101020097
S11374E000420102000029010000002A01000000FE
S11374F02B010000002C01000000340100000035C5
S113750001000000360100000043010200003A01BE
S11375100000003C010200003D010200003E0102A7
S113752000003F0102000044010200004501020086
S11375300046010200004701020000480102000069
S113754049010200004A010200004B010200004C04
S113755001020000370100000038010000002D0185
S11375600000002E010000002F0100000030010087
S113757000003101000000320100000000C00240A0
S113758000D0024000E00240F95C0000035D00000E
S11375900D5D00000000020001000000FFFFFF0F6E
S11375A0F486FF1F0000000000000000000000003F
S11375B000000000000000000000000000000000C7
S11375C000000000000000000000000000000000B7
S11375D000000000000000000000000000000000A7
S11375E00000000000000000000000000000000097
S11375F00000000000000000000000000000000087
S10776000000000082
S113760480B400AF094B5B78DBB25BB2002B07DBC1
S1137614064A064B5B78DBB263F07F03DBB253703C
S113762400BFBD465DF8047B704700BF0000024004
S113763480B500AF0121002000F056F8034B1B680D
S11376440133024A136000BF80BD00BF98140020B8
S113765480B500AF0221002000F046F8034B1B68FC
S11376640133024A136000BF80BD00BF9C14002094
S113767480B500AF0421002000F036F8034B1B68EA
S11376840133024A136000BF80BD00BF0084FF1FA2
S113769480B500AF0821002000F026F8034B1B68D6
S11376A40133024A136000BF80BD00BFA014002050
S11376B438B505460B4A137843F080031370144617
S11376C4237813F0800F05D1AB69B3F1FF3FF7D0F2
S11376D49847F5E7034B1B7813F0710F14BF01208F
S11376E4002038BD000002405FF800F0894B000020
S9030411E7
